:09000000021BF0024FFF25730002
:10000B00025135E4FFFE120750600C0FEF70010E2A
:0F001B0009E970F20A80EF220251445322E022D9
:07002B0002580A43EA4022DB
:1000330002791AEFC394094005EF940E4003BF20E1
:1000430003D38001C322244750524D430075A800B7
:100053009000E27406F09000E07480F09000E27487
:1000630012F002007D75A8009000E27406F0900083
:10007300E07400F09000E2740CF07455F5AE1238A1
:100083003578FFE4F6D8FD7581AA021C2E020456CA
:10009300E86480F8E933E83360110460F0ED33EC91
:1000A300337009E8FCE9FDEAFEEBFF220460DED3CE
:1000B300EB9FEA9EE99DE8C2E78CF0C2F795F0401A
:1000C3000CE8CCF8E9CDF9EACEFAEBCFFB12042128
:1000D30085D0F05804700320D5B3E80470075002AC
:1000E300B2D502046092D5EC0460F7E4CCC0E0C35F
:1000F30098F8603B94186008400DD0E0FB02043888
:10010300E4FBFAC9FC8028E830E406E4C9FBE4CA4E
:10011300FCE830E305E4C9CACBFCE854076010F8F7
:10012300C3E913F9EA13FAEB13FBEC13FCD8F13030
:10013300F52FC3E49CFCEF9BFFEE9AFEED99FDD0F7
:10014300E0FBEF4E4D4C701222DB0302045DEC2CFE
:10015300FCEF33FFEE33FEED33FDED30E7EB02044E
:1001630038EF2BFFEE3AFEED39FDD0E0FB50130BD9
:10017300BB0003020460ED13FDEE13FEEF13FFEC6F
:1001830013FC020438EC4D6011E8497017ED33ECB1
:100193003304600DE4FCFFFEFD22E933E833047011
:1001A300F802045612042158046009E4CC24815057
:1001B3000628500902046028400302045DC0E0EBF6
:1001C3004A7044B98006D0E0FB02044CEF4E701C29
:1001D300BD8008EBFFEAFEE9FD80EBE98DF0A4FEAC
:1001E300E5F0020271E9CDF9EAFEEBFFEF89F0A435
:1001F300FCE5F0CE89F0A42EFFE435F0CD89F0A420
:100203002DFEE435F08067EF4E7005BD80D780C3C7
:10021300EF8BF0A4ACF0EE8BF0A42CFCE435F0F8FB
:10022300EF8AF0A42CE5F038FCE433CB8DF0A42C5A
:10023300FCE5F03BF8EE8AF0A42CFCE5F038F8E49A
:1002430033CF89F0A42CFCE5F038CF3400CE89F00D
:10025300A42FFFE5F03EFEE433C98DF0A42EFEE5A6
:10026300F039CD8AF0A42FFFE5F03EFEE43DFD33E7
:10027300D0E0FB50070BBB000F020460EC2CFCEF3B
:1002830033FFEE33FEED33FD020438020460EC5D10
:10029300046005E85904700302045612042158044B
:1002A30060F6EC4860F2EC7004FDFEFF22C860DBF0
:1002B3002481C85009C3986002500602045D985017
:1002C300CAF582E9294B4A7005AB8202044C75F0EA
:1002D300007C1A7880C3EF9BEE9AED99400DC3EF33
:1002E3009BFFEE9AFEED99FDE842F0DC23ACF0D0E3
:1002F300E0FFD0E0FED0E0FDAB8220E7101BEB6017
:10030300BAEC2CFCEF33FFEE33FEED33FD02043881
:10031300E803F830E705C0F075F000EF2FFFEE3388
:10032300FEED33FD40B830E7C280AA74F8CC648098
:10033300CCC86480C8F582046043C3EB9FF5F0EA40
:100343009E42F0E99D42F0E89C45F060305018E58C
:10035300825FFFE582F42B5582FB50210ABA001D10
:1003630009B90019088016E5825BFBE582F42F5575
:1003730082FF50090EBE00050DBD00010CC3EB9FAB
:10038300F5F0EA9E42F0E99D42F0E89C45F06007F3
:10039300CC4820E701B3EC22ED33EC33600A047060
:1003A30003BD8004ECB2E7FC2275F020800E75F0EB
:1003B30010800575F0087D007E007F003392D530F4
:1003C300D503120978EC334010EF33FFEE33FEED23
:1003D30033FDEC33FCD5F0ED22E5F0247EA2D513FA
:1003E300CC92E7CDCEFF22EDD2E7CD33EC3392D5DD
:1003F30024814006E4FFFEFDFC22FCE4CFCECDCCFD
:1004030024E0501174FF80EDC3CC13CCCD13CDCEBB
:1004130013CECF13CF0470F030D5DE020978E9D2C2
:10042300E7C933E833F892D5EDD2E7CD33EC33FCAB
:100433005002B2D522EC30E7100FBF000C0EBE0005
:10044300080DBD00040BEB6014A2D5EB13FCED9279
:10045300E7FD2274FFFCFDFEFF22E480F8A2D574C1
:10046300FF13FC7D80E480EFC0E0EFFBEEFAEDF9D3
:10047300ECF8120188D0E0F5F0EFFBEEFAEDF9ECC1
:10048300F81209B6A3A3A3A3E8C0E0E9C0E0EAC059
:10049300E0EBC0E0C0F01201881209D3A3A3A3A329
:1004A300120097D0F0D0E0FBD0E0FAD0E0F9D0E032
:1004B300F8D5F0D4223F8000004120000042C8005C
:1004C30000447A0000461C400047C350004974248E
:1004D300004B1896804CBEBC205A0E1BCA6753C2F1
:1004E3001C749DC5AEFB60065407601C23231205D4
:1004F30016EB54386009120502120511120188EC3B
:10050300F8EDF9EEFAEFCB22EB12051180F1543836
:1005130003241C9004B8FE93FC0EEE93FD0EEE93A1
:100523000ECE93FF22F920E72824F950037907E43C
:10053300F42402FB18DBFDE624FB5014E9600DE410
:10054300F618E604F6B40A08E4F6D9F57401F60AD7
:1005530022C2D522ED33EC3392D5FA602AB4FF33AD
:10056300EDC2E77BFF60067A05797CE4227A0579A0
:100573008520D5047A057980224E614E002B494EA1
:1005830046002D494E4600E47A08F608DAFC7B0063
:10059300740722E8C0E0ECC0E0EDC0E0EEC0E0EF9D
:1005A300C0E0EA75F010A4CAABF075F04DA42BFBC4
:1005B300E435F0FCEA2410FAEB34C5FBEC34D9FC47
:1005C300EDC2E7FF75F056A4F42411C5F0F434C569
:1005D3008FF0A42AE5F03BE43CF620E7141204E88C
:1005E300D0E0FFD0E0FED0E0FDD0E0FC120291802D
:1005F30014F4041204E8D0E0FFD0E0FED0E0FDD014
:10060300E0FC120188D0E0F8E6FAEDD2E7CD33EC56
:10061300332482FBE4C3CF33CFCE33CECD33CD33BC
:10062300DBF37B0775F00A846004F6081B0AE5F028
:10063300F6088FF0740AA4FFACF08EF0740AA42CB1
:10064300FEACF050010C8DF0740AA42CFDE435F0DF
:10065300F608DBDE740722E709F608DFFA8046E7CF
:1006630009F208DFFA803E88828C83E709F0A3DF72
:10067300FA8032E309F608DFFA8078E309F208DF4B
:10068300FA807088828C83E309F0A3DFFA8064899F
:10069300828A83E0A3F608DFFA805889828A83E09E
:1006A300A3F208DFFA804C80D280FA80C680D4801F
:1006B3006980F28033801080A680EA809A80A880C7
:1006C300DA80E280CA803389828A83ECFAE493A3D6
:1006D300C8C582C8CCC583CCF0A3C8C582C8CCC565
:1006E30083CCDFE9DEE7800D89828A83E493A3F676
:1006F30008DFF9ECFAA9F0EDFB2289828A83ECFA90
:10070300E0A3C8C582C8CCC583CCF0A3C8C582C842
:10071300CCC583CCDFEADEE880DB89828A83E4937D
:10072300A3F208DFF980CC88F0EF60010E4E60C3BE
:1007330088F0ED2402B4040050B9F582EB2402B42E
:10074300040050AF23234582239006AA73BB0106FE
:1007530089828A83E0225002E722BBFE02E32289D8
:10076300828A83E49322BB010CE58229F582E58327
:100773003AF583E0225006E92582F8E622BBFE061D
:10078300E92582F8E222E58229F582E5833AF583B9
:10079300E49322BB010689828A83F0225002F72266
:1007A300BBFE01F322EF8DF0A4A8F0CF8CF0A428B8
:1007B300CE8DF0A42EFE22BC000BBE0029EF8DF0DF
:1007C30084FFADF022E4CCF875F008EF2FFFEE3391
:1007D300FEEC33FCEE9DEC984005FCEE9DFE0FD540
:1007E300F0E9E4CEFD22EDF8F5F0EE8420D21CFE14
:1007F300ADF075F008EF2FFFED33FD40079850067D
:10080300D5F0F222C398FD0FD5F0EA22C2D5EC3021
:10081300E709B2D5E4C39DFDE49CFCEE30E715B2D5
:10082300D5E4C39FFFE49EFE1207BAC3E49DFDE433
:100833009CFC80031207BA30D507C3E49FFFE49EF4
:10084300FE22A3F8E0C5F025F0F0E58215827002E0
:100853001583E0C838F0E822E88FF0A4CC8BF0A42D
:100863002CFCE98EF0A42CFC8AF0EDA42CFCEA8E7F
:10087300F0A4CDA8F08BF0A42DCC3825F0FDE98FA2
:10088300F0A42CCD35F0FCEB8EF0A4FEA9F0EB8F99
:10089300F0A4CFC5F02ECD39FEE43CFCEAA42DCE66
:1008A30035F0FDE43CFC2275F008758200EF2FFF64
:1008B300EE33FECD33CDCC33CCC58233C5829BED35
:1008C3009AEC99E58298400CF582EE9BFEED9AFD39
:1008D300EC99FC0FD5F0D6E4CEFBE4CDFAE4CCF9E9
:1008E300A88222B800C1B90059BA002DEC8BF0845C
:1008F300CFCECDFCE5F0CBF97818EF2FFFEE33FE2A
:10090300ED33FDEC33FCEB33FB10D703994004EBE1
:1009130099FB0FD8E5E4F9FA227818EF2FFFEE33AD
:10092300FEED33FDEC33FCC933C910D7059BE99ABF
:100933004007EC9BFCE99AF90FD8E0E4C9FAE4CC50
:10094300FB2275F010EF2FFFEE33FEED33FDCC33BA
:10095300CCC833C810D7079BEC9AE899400AED9BA3
:10096300FDEC9AFCE899F80FD5F0DAE4CDFBE4CC82
:10097300FAE4C8F922C3E49FFFE49EFEE49DFDE48C
:100983009CFC22EB9FF5F0EA9E42F0E99D42F0E8E1
:100993009C45F022E8600FECC313FCED13FDEE134E
:1009A300FEEF13FFD8F122E6FC08E6FD08E6FE0899
:1009B300E6FF22E493FC740193FD740293FE740337
:1009C30093FF22E6FB08E6F908E6FA08E6CBF822ED
:1009D300E493F8740193F9740293FA740393FB227A
:1009E300ECF608EDF608EEF608EFF622ECF0A3EDD0
:1009F300F0A3EEF0A3EFF022A42582F582E5F03513
:100A030083F58322FAE6FB0808E6F925F0F618E6F3
:100A1300CA3AF622D083D082F8E493701274019319
:100A2300700DA3A393F8740193F5828883E4737420
:100A330002936860EFA3A3A380DF8A838982E473B0
:100A4300EF4E6012EF60010EEDBB010B89828A83CA
:100A5300F0A3DFFCDEFA2289F05007F709DFFCA9D7
:100A6300F022BBFEFCF309DFFCA9F0220122000106
:100A73002000012300012100418810004488060062
:100A8300000000418811004188040041880F0041A3
:100A9300880D004188050041880200640080000041
:100AA3000000000000000000000000000000000043
:100AB3000000000000000000000000000000000033
:100AC3000000000000000000000000000000000023
:100AD3000000000000000000000000000000000013
:100E9300000000000000000000000000000000410E
:100EA30086210041851F00418520004487370000CB
:100EB30000004A874D000000000000000000004AC7
:100EC30087430000000000000000000044872D005D
:100ED30000000042872B00004487330000000041DC
:100EE30087310041875D004287200000418732003F
:100EF30042875B1C204487220000000041872900B1
:100F030041872A004187280044875E000000004192
:100F1300876300418764004187620044875700006C
:100F2300000044871C0000000044873F00000000CD
:100F330041872600418727004A879200000000006E
:100F4300000000FF004A879C000000000000000032
:100F5300FF004287A600004287B600004E87A80024
:100F6300000000000000000000000000004187B9FD
:100F7300004187B8004A88230000000000000000F9
:100F8300FF0042882D00004A882F00000000000067
:100F93000000FF0042883900004987C700050201AD
:100FA30005040205064987BE000502010504020582
:100FB300064187D1004187D0004287D20000418794
:100FC300D4005687D7000000005600000000000040
:100FD300000000000000FF0000000002A4862202BF
:100FE300A686224C87F51F1C1F1E1F1E1F1F1E1FB8
:100FF3001E1F41841B0002A8000041883B0041885A
:101003003CFF01AA0041883D0041883F0041883EE2
:101013000001240000E560244CF8E60560227849CD
:10102300302F02784CE475F001120A0702075020B2
:1010330028EB7F2ED2288018EF540F2490D434400D
:10104300D4FF302C0BEF24BFB41A0050032461FFEC
:10105300E561600215610564E56470020563302F84
:101063000D7849E475F001120A07EF020796021D95
:10107300FD7403D22F8003E4C22FF5608B498A4AA3
:10108300894BE4F561F563F564E56160077F201240
:10109300105380F57562FFC229C228C22AC22BC22F
:1010A3002DC22EC230121021FF700D302F057F008C
:1010B300121064AF64AE6322B4255FC2D5C22C1292
:1010C3001021FF24D0B40A00501A75F00A78613059
:1010D300D50508B6FF0106C6A426F620D50470027E
:1010E300D22B80D924CFB41A00EF5004C2E5D22CFE
:1010F300021351D22980C6D22880C0D22A80BCD202
:10110300D580BAD22D80B47F20121053202A0774C1
:1011130001B5610040F1121018FF12105302108C38
:10112300D230D22E8095121018FB121018FA12101A
:1011330018F94A4B700679487A147BFF202A2EE56A
:1011430061602A7E008E8275830012076960060E35
:10115300EE656270F0C2D5EBC0E0EAC0E0E9C0E042
:10116300EE1213B1D0E0F9D0E0FAD0E0FB12075051
:10117300FF60AAEBC0E0EAC0E0E9C0E0121053D080
:10118300E02401F9D0E03400FAD0E0FBE56204602A
:10119300DCD562D98087D22A80A212139460F7E546
:1011A30062700104120528A962600DE562600914EA
:1011B300F56212143BEF60F3EA30E702F404C399DB
:1011C3005077EAF425620430E701E404F562800D08
:1011D30012139460C1EA05622562120528EA785F5A
:1011E300F630E701E4256204D56204202D011412D0
:1011F30013B1E4C0E012143B785FE6601320E70705
:1012030014F612103B802204F6D0E014C0E07F00F5
:1012130012103BE56260071210321562800B302D0D
:1012230003121032D0E002108CD0E00480C51213F8
:101233009460A0E56204120528785FEAF6E562206F
:101243002D0260010424041213B174FF04C0E012E0
:10125300143B12103BE562202D026003121032D0C2
:10126300E0B562E87F45121045785FE67F2B30E7F3
:10127300047F2DF404C0E0121053D0E075F00A840B
:10128300C0F012103CD0E012103C02108C79108098
:10129300027908C22EC2308008D2D5790A80047937
:1012A3000AC2D5E562047002F562E4FAFDFEFF129C
:1012B3001018FC7B08202913121018FD7B1030280E
:1012C3000A121018FE121018FF7B20EC3382D592FD
:1012D300D55013C3E43028069FFFE49EFEE4202983
:1012E300039DFDE49CFCE4CBF8C229EC700CCFCE4B
:1012F300CDCCE824F8F870F38017C3EF33FFEE3357
:10130300FEED33FDEC33FCEB33FB994002FB0FD8CE
:10131300E9EB302905F8D0E0C448B229C0E00AEC73
:101323004D4E4F78207B0070C2EAB5620040BCC0CE
:10133300E01213B3D0F0D0E0202904C4C0E0C4B25B
:1013430029C0F012103CD0F0D5F0EB02108C120A39
:101353001711295312905810FA4C10F64212944F59
:10136300129C44129C49110F4312A25511D34612E9
:101373003145119D4714685010FE2D11022E112581
:101383002B11062311232014512A10BE48000011EB
:101393001DE562B4FF03756206121018FC121018E3
:1013A300FD121018FE121018FF7858020557790A1B
:1013B300A2D5202B14302D09B910020404B9080159
:1013C30004A2D5202E02500104202A68922AB56176
:1013D300005034C0E07F20302B197F30A22A722EB8
:1013E300722D500F12140AC22AC22EC22DC2307F90
:1013F30030800F302D03E9C0E0121053302D03D09D
:10140300E0F9D0E0B561CC302D177F30B9100C1264
:1014130010537F58302C077F788003B908031210CC
:1014230053302A057F2D0210537F202030F87F2B65
:10143300202EF322922A80CF7F00B4070050052488
:1014430058F8E6FF22286E756C6C2900D229121019
:10145300183029F8C229786130D50108F60210BE88
:101463002D504349581210182403B405004001E4D9
:1014730090146393121044743A121044D22B756182
:1014830004021290257300202573003E005F25732C
:101493000020202020202020202020202020202069
:1014A300004B4D4800253375004D5048003C005F0C
:1014B30025732020202020202020202020200025EC
:1014C30030337520004C41545F3A5F25635F25300C
:1014D3003375405F2530322E3032662720004C4F63
:1014E3004E5F3A5F25635F25303375405F253032A9
:1014F3002E3032662720004449525F3A5F2530334D
:1015030075400025336275005E0025733A20253649
:101513002E3166204D690025733A2025362E31661B
:10152300204B4D0025733A20252D322E316600566F
:101533000025733A202562782E25316278002573C1
:101543003A20002562752F2562752F2534750020FA
:101553004B204D204820284B4D2F482900204D205B
:1015630050204820284D494C452F482900474D54C9
:1015730020202B2562642000474D542020256264DF
:1015830020200025735F2573004D4F4455535F534F
:10159300454C45435449452020004C494D49455449
:1015A3002020202020202020202000474542525583
:1015B300494B45525350554E542020005645524CEA
:1015C30049434854494E472020202020004C414E97
:1015D30044494E5354454C4C494E472020005359DF
:1015E300535445454D494E464F202020202000208E
:1015F30045454E48454944202020202020202000F6
:101603002054494A445A4F4E452020202020202070
:10161300002042454C544F4F4E20202020202020B4
:101623002000FF72B2FF740FFF6563FF75D8FF5987
:1016330042FF3B8BFF73A8FF7560FF74EC257300BB
:1016430025336275005E004E4F253375004F20250C
:101653003375005A4F253375005A202533752A00F8
:101663005A57253375005720253375004E572533B8
:1016730075004E202533750025336C75004D002011
:101683002020203E002020203E3E0020203E3E3EE3
:1016930000203E3E3E3E003E3E3E3E3E0025735F02
:1016A3002020200025735F3E20200025735F3E3EEF
:1016B300200025735F3E3E3E00253475004D5048A3
:1016C300004B4D48004E4F25337540004F202533C6
:1016D3007540005A4F25337540005A202533754015
:1016E300005A572533754000572025337540004E67
:1016F3005725337540004E202533754000202020A8
:101703002020400025352E3166204D690025352ED9
:101713003166204B4D00253262753A2530326275B1
:10172300002573253262753A2530326275007E00DA
:1017330025362E3166204D690025362E3166204B25
:101743004D00253375204D504800253375204B4DF2
:10175300480025342E3166204D50480025342E3163
:1017630066204B4D4800253262752F253262750085
:1017730025733A252D322E316656004241540025F9
:10178300352E31664D690025352E31664B4D0025CA
:1017930033754D5048002533754B4D48002533753F
:1017A30000253275005175696E74657A7A00414C73
:1017B300455254455200475053202573002573204A
:1017C300257320212020003A70FA83BCAAE9E43E65
:1017D30081E0F8BF9DE9E63F80000039283C1ABB51
:1017E3009969663DA335E3BF255DE73FC90FDB413B
:1017F3008DDBCCC44936EE45C9913FC5B0F83D3FBA
:10180300800000C317F534452FFA73C60AFDDD12B5
:1018130018B904A2E192281420E0159017CA7404A1
:1018230012046B80261218B930E102B22820E0EBD3
:101833008C278D288E298F2A9017DE740412046B4F
:10184300A827A928AA29AB2A120188ED4C600730E2
:101853002804EC6480FC221218B9C0E08C278D2880
:101863008E298F2A901802740312046BA827A928C3
:10187300AA29AB2A120188ECC527FCEDC528FDEE89
:10188300C529FEEFC52AFF9017F2740312046BD02B
:1018930082A827A928AA29AB2AE58230E0071202E9
:1018A30091B22880A6EFCBFFEECAFEEDC9FDECC8CE
:1018B300FC1202918095ED33EC547FCC33922824B3
:1018C300605007D0E0D0E00204567B837AF9792296
:1018D300783E120188EDF933ECF83324815011EF8F
:1018E300FBEEFA1203EA1203ACECB2E7FC12009728
:1018F300ED33EC33602F2403F8C313FCED92E7FDC3
:10190300E82481E4501FECF8EDF9EEFAEFFB120343
:10191300EAEF04C2E0FCF5821203B6ECB2E7FC1274
:101923000097E58203FAED33EC3360071413FCED03
:1019330092E7FDEA22BE1249253E4CCCCDBEAAAAAF
:10194300AB3F8000003E7ADBB03EED63383F24BC02
:101953007D3F490FDBED33ECC2E7CC339228B4FF74
:1019630013ED547F60030204567FDB7E0F7DC97C39
:101973003F021A53C229C3947F401E7007EDD2E77A
:1019830094904015EFFBEEFAEDF9ECF87F007E0042
:101993007D807C3F120291D229ED33EC33248430D5
:1019A300E705E4C0E0806D04FAEDD2E754F0C333F9
:1019B300DAFD540734002323C0E0CCC0E0F8EDC0C7
:1019C300E0F9EEC0E0FAEFC0E0FBE41203B6EC246A
:1019D300FEFC8C388D398E3A8F3B1201887B007A5E
:1019E300007980783F120097ECC538B2E7FCEDC56B
:1019F30039FDEEC53AFEEFC53BFFD0E0FBD0E0FA80
:101A0300D0E0F9D0E0F8120097A838A939AA3AAB88
:101A13003B1202918C388D398E3A8F3B9019387472
:101A23000312046BA838A939AA3AAB3B120188D038
:101A3300E0600F2444F582E43419F5831209D312CC
:101A4300009730290B7BDB7A0F79C978BF12009797
:101A5300ED33EC336006ECA22892E7FC22C229C2E4
:101A63002AC22BC22CF9E4F52EF52FFCFDFEFFE96B
:101A73001028EA202B0CB42D04D22BD322B42B0232
:101A8300D32224D0504794095041240A302C15F80E
:101A9300852FF0740AA42872E74051C5F0704D8574
:101AA300F02FD322D22AC0E0E4FBFA792078411246
:101AB3000188ECF8EDF9EEFAEFFBD0E0FCE4120359
:101AC300B61200973029B4152ED322240A202C20D5
:101AD300B4FE0720291AD229D32224EB600424E080
:101AE300700EA22B9229D22CC22BD322C3020456EE
:101AF300E4302C0BE52F302B02F404A229922B3077
:101B03002AEA252E20D2E5A2E7922C5002F404B44F
:101B1300260050D8CCC0E0EDC0E0EEC0E0EFC0E05E
:101B2300EC1204E8D0E0FFD0E0FED0E0FDD0E0FC12
:101B3300202C051201888003120291302B0312031B
:101B43009BC32202045622EDA2E7D2E7F9EC33400D
:101B5300F260F3B4FF08ED547F70E8020460F824E8
:101B630081C2E0C0E0F40428FAC313FCED92E7FD60
:101B73008C308D318E328F33EEA2E7E9BA7F02C308
:101B83001334009400FA75F091A4E5F013F494FE75
:101B93008AF0A433E5F033248CD313FDE492E7FEFB
:101BA3007F007C3F758302ECC0E0F8EDC0E0F9EE06
:101BB300C0E0FAEFC0E0FBAC30AD31AE32AF331270
:101BC3000291D0E0FBD0E0FAD0E0F9D0E0F81200C7
:101BD30097ED6480FD30E7011CD583CBED33CC3327
:101BE300F8D0E0A2E71328C313CC13FD2202006848
:101BF30002364EE493A3F8E493A34003F68001F284
:101C030008DFF48029E493A3F85407240CC8C333F2
:101C1300C4540F4420C8834004F456800146F6DFC1
:101C2300E4800B0102040810204080900A6FE47ED8
:101C3300019360BCA3FF543F30E509541FFEE493B6
:101C4300A360010ECF54C025E060A840B8E493A37D
:101C5300FAE493A3F8E493A3C8C582C8CAC583CAA8
:101C6300F0A3C8C582C8CAC583CADFE9DEE780BE60
:101C73008F338E328D318C30AB37AA36A935A834E9
:101C83001202911219588F338E328D318C30E53414
:101C930030E747ECC0E0EDC0E0EEC0E0EFC0E0E4C9
:101CA300FFFEFDFCAB33AA32A931A83012032E7B11
:101CB300DB600250087A0F7949784080067A0F7901
:101CC3004978C0D0E0FFD0E0FED0E0FDD0E0FC12C8
:101CD30000978F338E328D318C30AF33AE32AD31CE
:101CE300AC30228B278A288929AB2AAA2BA92C124C
:101CF3000750FEAB27AA28A929120750FF6E702BA5
:101D0300EF600DE52E152E7002152D14452D700371
:101D13007F002274012529F529E43528F52874016B
:101D2300252CF52CE4352BF52B80BEAB27AA28A94F
:101D330029120750FFD3EE6480F8EF6480984003C4
:101D43007F01227FFF22D2288B2B8A2C892D121D03
:101D530085C0E0FF120036D0E040F3121A73400151
:101D630022ECC0E0EDC0E0EEC0E0EFC0E0121D8564
:101D7300D0F0AFF0D0F0AEF0D0F0ADF0D0F0ACF0EA
:101D830080D9E475F001782B120A070207502573F6
:101D9300005350454544005253002533754D504878
:101DA300002533754B4D48004C41534552003E3E90
:101DB3003E004B412042414E4400256264004B20CB
:101DC30042414E4400582042414E440085434C85D5
:101DD300444D85454EEBC546FBEAC547FAE9C54880
:101DE300F97F09784F120750F60809E970010ADFF5
:101DF300F4AB46AA47A948021074EFB40A07740D5E
:101E0300121E08740A309811A899B8130CC298309E
:101E130098FDA899C298B811F63099FDC299F59921
:101E23002225337500257300257331002573320095
:101E330025730025733A2575005F564F4C554D4564
:101E4300202020202020202020004750535F56458B
:101E53005242494E44454E00534E454C482E004194
:101E63004C41524D0041414E005549540043414DB0
:101E73004552410042494449524543542E00574577
:101E83004700434F4E54524F4C450045494E44453D
:101E9300004745564141524C2E004C4F4341544953
:101EA3004500574141525343482E0047454252553E
:101EB300494B45520050554E5400544F45474556E3
:101EC3004F45474400564F4C00474557495354002C
:101ED3004C45454700484F4F46444D454E55005FDE
:101EE3004D4F4455535F53454C454354494520207A
:101EF300004C494D494554005F5645524C494348AF
:101F030054494E472020202020004C414E44494E46
:101F13005354454C4C494E47202000535953544584
:101F2300454D494E464F2020202020005F45454E19
:101F330048454944202020202020202020005449C7
:101F43004A445A4F4E450042454C544F4F4E00426F
:101F5300454C544F4F4E005553455220494E464F22
:101F63000054455255475354454C4C454E00524935
:101F730054005354414E444141524400444554415A
:101F8300494C5300434F4D464F5254004A412000A1
:101F93004E4545004B4F4D504153004F444F004475
:101FA3004154554D00546563686E6F6C6F67696586
:101FB300005A454C4654455354004745454E20442A
:101FC30041544100545249502054494D4500424127
:101FD30054544552494A00534F46545741524500C1
:101FE3004441544142414E4B004F504745534C41AD
:101FF30047454E004745425255494B45525350556C
:102003004E54454E00522F4F444F0047454D005408
:10201300494A440000000000000000004F4F000048
:1020230000060006000000487A410000F825252438
:10203300F800007F25251A007D4140417D00000006
:10204300000B070000487A490000F824252525F8ED
:1020530003030000000008083E08080000000058C1
:10206300380008080808080000004000000020109D
:10207300080402003E5149453E0000427F400000F3
:102083004261514946002241494936001814127FE2
:1020930010002745454539003C4A49493000017144
:1020A30009050300364949493600064949291E00F6
:1020B300003636000000005B3B00000000081C3EB9
:1020C3007F001414141414007F3E1C080000020146
:1020D30059090600324959413E007E1111117E0013
:1020E300417F494936003E4141412200417F414100
:1020F3003E007F49494141007F09090901003E41F2
:1021030049497A007F0808087F0000417F410000A9
:102113002040413F01007F08142241007F4040409E
:1021230040007F020C027F007F0204087F003E41D3
:1021330041413E007F09090906003E4151215E00ED
:102143007F091929460026494949320001017F01C7
:1021530001003F4040403F000718601807003F4020
:1021630038403F0063140814630007087008070031
:10217300615149454300007F4141000002040810BA
:1021830020000041417F000004020102040040409E
:1021930040404000000402010000205454547800E1
:1021A3007F48444438003844444420003844444879
:1021B3007F00385454540800087E090200000814B4
:1021C30054543C007F080404780000447D40000020
:1021D3002040443D0000007F1028440000417F4020
:1021E30000007804180478007C080404780038445C
:1021F300444438007C14242418001824147C400020
:10220300007C08040400485454542000043E442035
:1022130000003C4040207C001C2040201C003C402F
:1022230030403C004428102844004C5050503C009F
:102233004464544C44000008364100000000770019
:1022430000000041360800000804081008002A5561
:102253002A552A00080000000000000000000000CA
:1022630000000000000400F8F800000D0D0006381F
:1022730038003838000000000000000820F8F8207B
:10228300F8F82000020F0F020F0F0200003078CE83
:102293008E18100000040C38390F060008183C246F
:1022A300BCD86030000006030E1E121E0C0800B0DE
:1022B300F8487830000000070F0809070F090238B3
:1022C30038000004E0F81C04030F1C1004041CF87D
:1022D300E0101C0F030780A0E0C0E0A08000020311
:1022E30001030200068080E0E08080000003030019
:1022F30000030000002C3C1C06808080808080004E
:1023030000000000000400000000000C0C000600A8
:1023130000C0F03C0C0C0F030000000800F0F808AC
:1023230068F8F00000070F0B080F070008002020D3
:1023330030F8F80000000000000F0F000008003024
:10234300380888F87000000C0E0B09080800080014
:1023530030388888F8700000060E08080F07000858
:102363000000F8F800E0E00000030302020F0F0290
:102373000800F8F88888880800000808080C070394
:10238300000800C0E07858C8800000070F08080F55
:1023930007000800080888E878180000000E0F01FD
:1023A300000000080070F8C888F8700000070F08E4
:1023B300090F07000800F0F80808F8F0000000090A
:1023C3000D0F030100080000006060000000000022
:1023D300000C0C000000080000006060000000001A
:1023E30000002C1C000000070080C0E0F0F8000093
:1023F300000103070F000560606060000C0C0C0C0B
:10240300000700F8F0E0C08000000F0703010000A0
:102413000760701090F0600000001B1B00000004B8
:1024230000382838000000000800E0F01818F0E039
:1024330000000F0F01010F0F000800F8F88888F85B
:102443007000000F0F08080F07000800F0F80808D5
:1024530038300000070F08080E06000800F8F808D7
:1024630018F0E000000F0F080C0703000800F8F84D
:102473008888880800000F0F08080808000800F87B
:10248300F88888880800000F0F000000000008008B
:10249300F0F8080838300000070F08090F0F00088C
:1024A30000F8F88080F8F800000F0F00000F0F000D
:1024B30008000008F8F80800000000080F0F0800E3
:1024C30000080000000000F8F80000060E08080FDE
:1024D30007000800F8F880E0781800000F0F0003E9
:1024E3000F0C000800F8F80000000000000F0F08B0
:1024F300080808000800F8F820C020F8F8000F0FBB
:102503000001000F0F0800F8F860C080F8F8000F12
:102513000F0000010F0F0800F0F80808F8F00000A2
:10252300070F08080F07000800F8F88888F87000FC
:10253300000F0F00000000000800F0F80808F8F092
:102543000000070F08181F17000800F8F88888F81C
:102553007000000F0F00010F0E0008003078C888CC
:1025630018100000040C08090F060008000808F8FA
:10257300F80808000000000F0F0000000800F8F83A
:102583000000F8F80000070F08080F07000800F81C
:10259300F80000F8F8000003070C0C07030008001C
:1025A300F8F800C000F8F800010F0E010E0F010843
:1025B300001838E0C0381800000E0F00010F0E009D
:1025C300080078F88080F878000000000F0F000002
:1025D300000800080888C8783800000E0F090808AA
:1025E30008000404FCFC00101F1F000638F8C0009C
:1025F30000000000030F0C0004FCFC04001F1F106C
:1026030000080C1E92DE6C301800000301060F094F
:102613000F0604000000000000000004000000009A
:10262300000000000800F2FA1818FAF200000F0F79
:1026330001010F0F000800FAFA0000FAFA00000780
:102643000F0C0C0F07000800F2FA0808FAF200005A
:10265300070F08080F07000800F0FA1A19F9F0002D
:10266300000F0F01010F0F000800F8FA8A8989088B
:1026730000000F0F08080808000800080AFAF90903
:1026830008000008080F0F0808000800F0FA0A09FC
:10269300F9F00000070F08080F07000800F8FA0216
:1026A30001F9F80000070F08080F07000800FAF9FE
:1026B300C382F9F800000F0F00010F0F000800F8A4
:1026C300FA0101FAF80000070F0C0C0F07000800CD
:1026D300F8F9898A8A0800000F0F0808080800081B
:1026E300000809F9FA0A08000008080F0F08080093
:1026F3000800F0F9898AFAF000000F0F01010F0FAB
:10270300000800F8044444788000000F000202022D
:1027130001000800C0E02020E0C00000070F080807
:102723000F07000800E0E02020E0C000003F3F0862
:10273300080F07000800C0E02020E0E00000070FBA
:1027430008083F3F000800E0E08040606000000FA1
:102753000F00000000000800C0E02020202000003F
:10276300080909090F0600080020F8F820202000B6
:102773000000070F080808000800E0E00000E0E0A0
:102783000000070F08080F0F000800E0E00000E05A
:10279300E0000003070C0C0703000800E0E000C0A2
:1027A30000E0E000030F0C030C0F03080060E0805F
:1027B30080E06000000C0E03030E0C000800E0E054
:1027C3000000E0E000002327341C0F03000800F999
:1027D300F98A8A8A0800000F0F0808080800FF22F8
:1027E30057FF2268FF2271FF227EFF228FFF229F65
:1027F300FF22B0FF22C1FF22C6FF22CFFF22D8FF54
:1028030022E7FF22F4FF22FBFF2308FF2311FF230C
:102813001EFF232FFF2340FF2351FF2362FF237358
:10282300FF2384FF2395FF23A6FF23B7FF23C8FFBE
:1028330023D9FF23EAFF23F9FF2404FF2413FF24F2
:1028430022FF242BFF243CFF244DFF245EFF246F33
:10285300FF2480FF2491FF24A2FF24B3FF24C4FF9D
:1028630024D5FF24E6FF24F7FF2508FF2519FF25BC
:102873002AFF253BFF254CFF255DFF256EFF257FA6
:10288300FF2590FF25A1FF25B2FF25C3FF25D4FF18
:1028930025E5FF25EEFF25FBFF2604FF2615FF2672
:1028A3001EFF2627FF2638FF2649FF265AFF266BE1
:1028B300FF267CFF268DFF269EFF26AFFF26C0FF47
:1028C30026D1FF26E2FF26F3FF2704FF2715FF2764
:1028D30026FF2737FF2748FF2759FF276AFF277B54
:1028E300FF278CFF279DFF27AEFF27BFFF27D00CB5
:1028F300F0F8FCFEFE0E8EFEFEFCF8F0FFFFFFFF7D
:10290300FFF81FFFFFFFFFFF0F1F3F7F7F70707FE9
:102913007F3F1F0F0C000070707078FCFCFEFEFE02
:1029230000000000000000FFFFFFFFFF00000000A9
:102933000000007F7F7F7F7F000C00F0FCFCFE0E19
:102943000EFEFEFCF8F000000080E0F8FEFFFF3F03
:102953001F0300787E7F7F7F7F73707070000CF0A1
:10296300FCFCFEFE0E0EFEFEFCFCF0C1C1C1C1DD8F
:102973001C3CFFFFFFF7E30F3F3F7F7F70707F7FBC
:102983003F3F0F0C000080F0FE3EFEFEFEFE000007
:10299300E0FCFFDFC3C0FFFFFFFFC0C0070707075F
:1029A30007077F7F7F7F07070CFEFEFEFEFE0E8E6E
:1029B3008E8E8E0E0E8F8F8F8F8F0303FFFFFFFF81
:1029C300FE0F3F3F7F7F70707F7F3F3F0F0CF0F81C
:1029D300FCFEFE0E0E7E7E7C7C70FFFFFFFFFF067B
:1029E30007FFFFFFFEFC0F3F3F7F7F70707F7F3F3E
:1029F3003F0F0C001E1E1E1E1E1EFEFEFEFEFE00D0
:102A0300000000E0F8FFFFFF1F07000060787F7FF2
:102A13007F1F07000000000CF0FCFCFEFE0E0EFE04
:102A2300FEFCFCF0E3F7FFFFFF1C1CFFFFFFF7E3D7
:102A33000F3F3F7F7F70707F7F3F3F0F0CF0FCFCA9
:102A4300FEFE0E0EFEFEFCF8F03F7FFFFFFFE06090
:102A5300FFFFFFFFFF0E3E3E7E7E70707F7F3F1FB6
:102A63000F02707000000E0E020C040CFEFEFCF848
:102A7300F0E0C08000000000FFFFFFFFFFFFFFFF4B
:102A8300FF7E3C187F7F3F1F0F07030100000000FC
:102A93000E040C1E1E0C00000000000000000E00BF
:102AA300C0FEFEFEFE1EFEFEFEFEC00000E0FFFFB7
:102AB300FFFF878087FFFFFFFFE0007F7F7F7F07A8
:102AC300070707077F7F7F7F000CFEFEFEFEFE1ECB
:102AD3001EFEFEFCFCF0FFFFFFFFFF1E1EFFFFFBC1
:102AE300FBF17F7F7F7F7F78787F7F7F3F1F0DF0B4
:102AF300F8FCFCFE1E1E1EFEFEFCF8F0FFFFFFFFAF
:102B0300FF000000E3E3E3E3E30F1F3F7F7F7878F9
:102B1300787F3F3F1F070CFEFEFEFEFE1E1EFEFEDD
:102B2300FCFCF8FFFFFFFFFF0000FFFFFFFFFF7F3D
:102B33007F7F7F7F78787F7F7F3F1F0BFEFEFEFEC8
:102B4300FE1E1E1E1E1E1EFFFFFFFFFF3C3C3C3CE5
:102B53003C007F7F7F7F7F7878787878780BFEFEE4
:102B6300FEFEFE1E1E1E1E1E1EFFFFFFFFFF3C3C41
:102B73003C3C3C007F7F7F7F7F0000000000000C17
:102B8300F0F8FCFEFE1E1EFEFEFCF8F0FFFFFFFF4A
:102B9300FF0038F9F9F9F9F90F1F3F7F7F78787F44
:102BA3001F7F7F7F0DFEFEFEFEFE000000FEFEFE89
:102BB300FEFEFFFFFFFFFF3C3C3CFFFFFFFFFF7FED
:102BC3007F7F7F7F0000007F7F7F7F7F05FEFEFE8C
:102BD300FEFEFFFFFFFFFF7F7F7F7F7F0800000078
:102BE300FEFEFEFEFE000000FFFFFFFFFF78787889
:102BF3007F7F7F3F1F0DFEFEFEFEFE00C0F8FEFE40
:102C0300FE3E06FFFFFFFFFF7FFFFFFFF780000091
:102C13007F7F7F7F7F00030F7F7F7F7C700AFEFEB5
:102C2300FEFEFE0000000000FFFFFFFFFF000000AC
:102C330000007F7F7F7F7F787878787811FEFEFEB3
:102C4300FEFEFEFEE000E0FEFEFEFEFEFEFEFFFFD9
:102C5300FFFFFF00FFFFF8FFFF00FFFFFFFFFF7F06
:102C63007F7F7F7F00037F7F7F03007F7F7F7F7F67
:102C73000CFEFEFEFEF88000FEFEFEFEFEFFFFFFE2
:102C8300FFFF1FF8FFFFFFFFFF7F7F7F7F7F0001B5
:102C93001F7F7F7F7F0CF0F8FCFEFE1E1EFEFEFCF6
:102CA300F8F0FFFFFFFFFF0000FFFFFFFFFF0F1F15
:102CB3003F7F7F78787F7F3F1F0F0CFEFEFEFEFE77
:102CC3001E1EFEFEFEFCF8FFFFFFFFFF3C3C3F3FE6
:102CD3003F1F0F7F7F7F7F7F000000000000000CFD
:102CE300F0F8FCFEFE1E1EFEFEFCF8F0FFFFFFFFE9
:102CF300FF0000FFFFFFFFFF0F1F3F7F7F78F8FFFD
:102D0300FFDFDFCF0CFEFEFEFEFE1E1EFEFEFEFC00
:102D1300F8FFFFFFFFFF1E1EFFFFFFF7E37F7F7F2D
:102D23007F7F00007F7F7F7F7F0DF0FCFCFEFE1E18
:102D33001EFEFEFCFCF80083878F9F9F3F7F7EFC77
:102D4300F8F8F0C00F1F3F7F7F7878787F7F3F3F91
:102D53000F0C1E1E1EFEFEFEFEFEFE1E1E1E0000AD
:102D630000FFFFFFFFFFFF0000000000007F7F7FE9
:102D73007F7F7F0000000CFEFEFEFEFE0000FEFED5
:102D8300FEFEFEFFFFFFFFFF0000FFFFFFFFFF0F41
:102D93001F3F7F7F78787F7F3F1F0F0F151EFEFE3B
:102DA300FEFEC00000FEFEFEFEFE0000C0FEFEFEB4
:102DB300FE1E001FFFFFFFFF00FFFFFF03FFFFFFDC
:102DC30000FFFFFFFF1F0000001F7F7F7F7E7F7FCD
:102DD3000100017F7F7C7F7F7F1F00000D063EFE89
:102DE300FEF8E000C0F8FEFE3E060000C0FFFFFF55
:102DF3003FFFFFFFC00000707E7F7F1F0100011FA8
:102E03007F7F7E700D0A001E1E1EDEFEFEFEFE7E0E
:102E13000080F0FEFFFFFF1F0300787F7F7F7F7F2F
:102E230078787878FF28F2FF2917FF293CFF29617A
:102E3300FF2986FF29ABFF29D0FF29F5FF2A1AFFB7
:102E43002A3FFF2A64FF2A6BFF2A6CFF2A6DFF2AA1
:102E53006EFF2A93FF2A94FF2AA1FF2ACCFF2AF1AF
:102E6300FF2B19FF2B3EFF2B60FF2B82FF2BA7FFAE
:102E73002BCFFF2BDFFF2BF8FF2C20FF2C3FFF2C4A
:102E830073FF2C98FF2CBDFF2CE2FF2D07FF2D2C89
:102E9300FF2D54FF2D79FF2D9EFF2D9FFF2DDFFF6B
:102EA3002E07FF2E080B013C24242424242424244D
:102EB3003C000B013C3C3C3C3C3C3C3C3C3C000A65
:102EC3000200FE020202020202FE00007F404040B6
:102ED3004040407F000A0200FEFEFEFEFEFEFEFEB4
:102EE30000007F7F7F7F7F7F7F7F001002000000D5
:102EF30000C0F0FC1E1EFCF0C000000000C0F0FC8F
:102F0300FFFFFFFFC8C8FFFFFFFFFCF0C01E040068
:102F130000000000C0C00000181800001F020408D1
:102F23001F000018180000C0C000000000C000808F
:102F33000CCC0000000000000000000000000000B6
:102F4300000000000000804C4C40800304076463D1
:102F5300000000000000000000000000000000006E
:102F63000000000003646404030000000000000686
:102F7300060030300000C8A8A898000030300000D8
:102F830006060000000000100200000080E0F8FECA
:102F9300FFFEF8E0800000000060783E3F1F1F0F37
:102FA3000F0F1F1F3F3E7860001002030F3EFEFC11
:102FB300FCF8F8F0F0E0E0C0C0800060783E3F1F0E
:102FC3001F0F0F07070303010100001002030F3E49
:102FD300FEFCFCF8F8F8FCFCFE3E0F0300000000CA
:102FE30000030F3F7F3F0F0300000000001002802B
:102FF300C0C0E0E0F0F0F8F8FCFCFE3E0F03000078
:103003000101030307070F0F1F1F3F3E78600010E6
:103013000200008080C0C0F0FCFFFFFCF0800000D5
:1030230000030307070F0F0F1F1F1F3F3F7F7C7016
:10303300801002C0C0E0E0F0F0F0F8F8F8FCFCFE0D
:103043003E0E010000010103030F3FFFFF3F0F018D
:103053000000001002010E3EFEFCFCF8F8F8F0F050
:10306300F0E0E0C0C0000000010F3FFFFF3F0F038F
:103073000301010000100200000080F0FCFFFFFCD0
:10308300F0C0C08080000000707C7F3F3F1F1F1F87
:103093000F0F0F07070303200400000000000000C8
:1030A300000080C0E0F0F8FCFEFCF8F0E0C0800017
:1030B3000000000000000000000080C0E0F0F8FC09
:1030C3001E1FFF0FFF03132B13030303030303FF4E
:1030D300FEFCF8F0E0C080000000000103070F1FB2
:1030E3003C7CF1F0F7E0E0E0E0E0E6E9E9E6E07FF0
:1030F3003F1F0F0703010000000000000000000055
:103103000000000103070F1F3F1F0F07030100000B
:103113000000000000000000002004000000000088
:103123000000000080C0E0F0F8FCFEFCF8F0E0C016
:1031330080000000000000000000000080C0E0F0FC
:10314300F8FC1E1F0FFF03132B13030303030303D7
:10315300FF0F1E1CF8F0E0C0800000000001030711
:103163000F1F3C7CF0F7E0E0E0E0E0E6E9E9E6E0B1
:10317300F7703C1C0F070301000000000000000073
:1031830000000000000103070F1F3F1F0F0703018B
:103193000000000000000000000000200400000008
:1031A30000000000000000000000C0F0F8F8F0C0CC
:1031B300000000000000000000000000000000000C
:1031C300000000000000C0F0FCFFFF03030303FF47
:1031D300FFFCF0C000000000000000000000000041
:1031E3000000C0F0FCFFFFFFFFFFFF60606060FFB7
:1031F300FFFFFFFFFFFCF0C0000000000000000025
:1032030000070F0F0F0F0F0F0F0F0F0C0C0C0C0FEE
:103213000F0F0F0F0F0F0F0F07000000001803FC15
:1032230002010101010181C1E1F1F9F9F1E1C1817A
:10323300010101010102FCFF00000004060707076A
:10324300FFFFFFFFFFFF0707070604000000FF3F24
:1032530040808080808080809F9F9F9F9F9F8080F1
:103263008080808080403F1803FC02010101E1E17E
:10327300E1E1E1E1E1E1E1E16121010101010102BA
:10328300FCFF00000000FFFF7F3F3F7FFFFFFFFCCD
:10329300F8F0E0C080000000FF3F40808080818024
:1032A30080808080808183878F8F87838180804027
:1032B3003F1803FC02010101010181C1E1F1010198
:1032C30001010101010101010102FCFF0000183CA1
:1032D3007EFFFFFFFFFF7E7E7E7E7E7E7E7E7E7E86
:1032E3000000FF3F4080808080808183878F8080C3
:1032F300808080808080808080403F1803FC0201B2
:1033030001010101010101010101F1E1C18101019A
:1033130001010102FCFF00007E7E7E7E7E7E7E7EBA
:103323007E7EFFFFFFFFFF7E3C180000FF3F4080D3
:10333300808080808080808080808F878381808070
:10334300808080403F1803FC0201010101012161DB
:10335300E1E1E1E1E1E1E1E1E1E101010102FCFFA0
:1033630000000080C0E0F0F8FCFFFFFF7F3F3F7FDD
:10337300FFFF00000000FF3F4080808183878F8F25
:1033830087838180808080808081808080403F0728
:10339300011C22514945221C300600000000000098
:1033A3000080C0E0E0F0F8F8FC7C7E3E3E3E3E3F0D
:1033B3001F1F1F1F1E3E3E3E3E7C7CFCF8F8F0E0C4
:1033C300E0C080000000000000000000C0F0F8FE34
:1033D300FF7F3F0F07030101000000000000000012
:1033E300000000000000000080C0E0F0F9FDFF7F56
:1033F3003F3F7FFFFEF8F0C00000E0FFFFFFFF3F0D
:1034030001000000000000000000000000000000B8
:1034130080C0E0F0F8FCFE7F3F1F0F0703010000B0
:10342300000000013FFFFFFFFFE0037FFFFFFFF806
:10343300800000000000000080C0E0F0F8FCFE7F88
:103443003F1F0F0703010000000000000000000001
:1034530000000080F8FFFFFF7F030000030F1F7FC2
:10346300FFFEFCF0F8FCFEFF3F1F0F070301000007
:103473000000000000000000000000008080C0E0A9
:10348300F0FCFEFF7F1F0F030000000000000000A0
:1034930000010307070F1F1F3F3E7E7C7C7C7CFCE3
:1034A300F8F8F8F8787C7C7C7C3E3E3F1F1F0F07C2
:1034B3000703010000000000000010010000007C71
:1034C30092107C4444447C10927C00002004000051
:1034D3000000000000000000000000FCE282020285
:1034E3000404080810A040A010080606000000000D
:1034F3000000000000000000000000FFFFFFFEFCD2
:10350300F8F8E4C28100000001020C30C0000000A2
:103513000000000000000078FCFEFFFFFFCF8707DC
:10352300070707070707070606040404030000004C
:1035330000183C3C3C3C3C3C3C3D3F3F3F3F3F3F15
:103543003E3C3C3C3C3C3C3C3C3C180000001201F3
:1035530010010000000883040000000101020001C3
:1035630009092100010001222E00090222000101A4
:1035730000C0FA0904000001030000000921000152
:103583000001222E000705810308006400002E06B7
:10359300A0FF09A5A10109A609A51580257F750826
:1035A3009540B10209A71580257F7508950881020A
:1035B30009A91580257F750895409102C004030968
:1035C300041A03570049004C004C002000540052D9
:1035D300004E004900430053000000180347005009
:1035E300005300200041004C0045005200540045A8
:1035F300005200FF35C0FF35C4FF35DE0099A3AD8F
:10360300B8C2CCD6E0EBF500919293949597999B31
:103613009EDE00000000000000000000000000002B
:1036230000F12C1248761260BF1248001271681222
:103633007149E4F522F523F521F5249087B9F0D2F9
:103643000C90880D04F0F1F5020026D124124D539D
:103653001251A8EF640A706B125252EF604924FAB8
:103663007061126FFB12493C9087A6E07002A3E0E1
:103673007003124A2B900013E054FDF0A20DB39295
:103683000D90875BE07002A3E06002F1C69087A60D
:10369300E07002A3E0600890879BE0FF124E872052
:1036A3001921124E0C801C900013E06402F0127179
:1036B300A81271D912433090875BE07002A3E060D7
:1036C30002F1C6F1F5300828201A25201B22201C00
:1036D3001F201D1C201E19201F16C39087E7E0948E
:1036E3001E9087E6E094004005124BF18002C22051
:1036F30030082020201D201A1A201B17201C1420FC
:103703001D11201E0E201F0B124F3B90880BE0FF54
:10371300126A781248DB125C06123B6F90841BE03E
:103723007002C153F1DD020050902000E0F520301B
:10373300004AE4908803F09088127405F090880E94
:103743007409F0E490880AF090880BF090880C7468
:103753000CF0C201C202C200F1E77C207F011240DB
:10376300957D007C607F03123ABD90880AE0FB7D63
:1037730005123AF8F1D5123AF8123F3F902000E0D3
:10378300F520A3E0908803F0902002E0908812F0E7
:10379300902003E090880EF0902004E090880BF0D6
:1037A300902005E090880AF0902006E090880CF0C5
:1037B300783B7C877D017B017A6079007E007F0402
:1037C30002072A90875CE024FFF090875BE034FFD8
:1037D300F02290880CE0FB7D0622E47F107E27FD1B
:1037E300FC024DCAE4FFFEFDFC90873B1209EF7D0E
:1037F3000022300C3C90880DE025E025E04422F5C2
:1038030097E59730E0FB90880DE0FF1460080470A3
:103813000B9088058003908802E596F0EFC394012E
:10382300500890880DE004F08005E490880DF0C204
:103833000C22E4900005F0900003F090000774FF61
:10384300F0E4900009F09000137407F090001574F1
:1038530002F090001714F09000B07438F09000B4A8
:103863007430F09000C77401F0228C6F8D70E4FE09
:10387300F9BF0105127CD98011BF0205127CC980F2
:1038830009BF0304F1D9800251AD74A0F011DEEB3E
:10389300F053038011DEE0F1F8B503047E018005E7
:1038A300BC20027901EE7003EC60E9E96401702841
:1038B30011DEE05480B503027E01BF01059025555A
:1038C3008013BF0205904555800BBF0305906555D6
:1038D300800390855574F0F0AF0622857082856F62
:1038E30083228F658B688A69896ACEECCECFEDCF50
:1038F3008E6D8F6EE56C156CAE6B7002156B4E6042
:103903002E127CC07002056914F9120750FBAD6ECC
:10391300AC6DAF65116D056EE56EAE6D7002056D34
:1039230014F5828E83E0FF908461E02FF080C5223E
:1039330090849EE0600221C490841CE024FD600218
:1039430021C490849DE0FE7032EFD394014072EF66
:1039530024FFFDE434FFFC908420E0FAA3E0FBC3E2
:103963009DEA9C5008CCEACCCDEBCD8004EF24FF3C
:10397300FD789EEDF6EE0408F6801BEFFDC3908400
:1039830021E09D31C55005A3E0FF8000789EEFF64E
:1039930090849DE008F690841D127C2F789FE62486
:1039A3009EF9E43484FA7B0118E6756B00F56C111B
:1039B300E5789E127D34700990841CF0A3E0FF51DA
:1039C3009022908420E09400228F6590849CE06094
:1039D30037E5656002418F90845C7405F090841C28
:1039E300E090845DF09000E0E090845EF09000E26F
:1039F300E090845FF078DF7C847D017B017A8479B9
:103A03005C7E007F4002072A90841CE024FC705EE9
:103A1300E5657020C3908421E0940731C55005A368
:103A2300E0FF80027F07789EEFF6756501E49084DE
:103A3300DFF08016C3908421E0940831C55005A3BC
:103A4300E0FF80027F08789EEFF690841EE0FEA3DD
:103A5300E0FF74DF2565127C1F789EE6756B00F529
:103A63006C127C8F127D34702390841CF022E478D6
:103A73009FF6789FE6FFC394085011E5652F24DF76
:103A8300F582E43484F583E4F00680E622BF010581
:103A9300127CD98011BF0205127CC98009BF0304BF
:103AA300F1D9800251AD74F0F02290855574AAF0DB
:103AB300908AAA7455F090855522124095AB207DCB
:103AC300007C207F0151FC908803E0FB7D017C207A
:103AD3007F0151FC908812E0FB7D027C207F015125
:103AE300FC90880EE0FB7D037C207F0151FC9088D5
:103AF3000BE0FB7D047C207F018C298D2AE4FEF9F9
:103B0300BF0105127CD98011BF0205127CC980094F
:103B1300BF0304F1D9800251AD74A0F0852A8285D8
:103B23002983EBF0530380F1F0F1F8B503047E0130
:103B33008005BC20027901EE7003EC60EAE96401C0
:103B43007027F1F05480B503027E01BF0105902573
:103B5300558013BF0205904555800BBF0305906543
:103B630055800390855574F0F0AF06223009187D17
:103B7300007C207F0151BD90880AE0FB7D0551F850
:103B83001237D551F8C20922E47872F6301102A136
:103B93003A90841BE06002A13A124F3B1274DA752B
:103BA300321F75331EE4FB1258ED125FFA12714097
:103BB3004401F0D2AF1237F5300119752EFF752F7E
:103BC3001575300D127EC9126EEB90873BF13312DF
:103BD3006EFE8014752EFF752F1575301A127EC96F
:103BE30090873BF133126F521266BA7B027D03E476
:103BF300FFB1507872E664017BFF7A1F798F7029D9
:103C0300F184127E89B1507BFF7A1F798F126FD7AF
:103C1300FFC3743A9FFF752A017B3A7D0312603814
:103C2300F192127E45B1508024F184127E89F17E97
:103C3300F195127E45B1507BFF7A1F7993126FD7AE
:103C43002443FB752A017D037F43126038752EFFE1
:103C5300752F157530277531FF75321F7533D112E6
:103C630066A67B047D03E4FFF17EF195753215753D
:103C730033327B047D58E4FFF17E752F15753034A4
:103C83007531FF75321F7533DA907FFFE493FFC4FC
:103C9300540FF534EF540FF5357B057D03E4FFF145
:103CA3007E752F157530417531FF75321F7533E3FE
:103CB3007B067D03E4FFF17E752F157530469080FA
:103CC300001209B67811120997EF541FFFE48F31E0
:103CD3001209B67816120997EF540FFFE48F3212C8
:103CE30009B6781A120997EF543FFFEF24D0F53441
:103CF300E43407F5337B067D3FE4FFB1503012080F
:103D0300E47872F6C212800930130678727601C223
:103D130013A210E433FF7872E67E00B401027E0141
:103D2300EE5F600E1237E77C607F03124095F13F30
:103D3300C2101248DB618F22752F1E753028753132
:103D4300FF75321E7533857B027D1E7F018F2B8DA0
:103D53002C8B2DE4908767F0A3F0A3F0A3F0787584
:103D6300762E087627F540754100754231852E433E
:103D7300852F448530458540468541478542487BAC
:103D8300017A847902121DCFF1CAFF7002C1DBE50B
:103D93002B705EEF24E0908769F0A37406F0E4A330
:103DA300F0F19F4002C1C8908768E0FDE52C2DFD2E
:103DB300E433FCEE7E002DFFEE3C127EB44002C1E4
:103DC300C890876BE0F9908769E075F006A4241723
:103DD300F582E5F03420F583E58229124760E49308
:103DE300FD75F080E52D1247A01247EEEDF1B3808B
:103DF300B0E52B64017041F1CA24E0127F4F24E146
:103E0300F582E5F03427127D11E490876BF0F19F82
:103E1300501E127D7B5019127DCEF1E9C083C08202
:103E230090876BE0FFD082D083124776F1AA80DEC1
:103E3300F1C2640270D3C1C8E52B64026002C1C839
:103E4300F1CAFF64206047EF24D0127F4F2427F587
:103E530082E5F0342E127D11E490876BF0F19F50D0
:103E63001E127D7B5019127DCEF1E9C083C0829072
:103E7300876BE0FFD082D083124776F1AA80DEF110
:103E8300C2640370D390876AE02402F0803790877E
:103E93006A740E127D2DE490876BF0F19F5021EE32
:103EA300252CFFE433FE908768E07C002FFFEC3E77
:103EB300127EB4500B1247971247EEE4F1B380DB46
:103EC300F1C2B403D190876AE0FF908768E02FF0D6
:103ED300908767E004F0A18BE52B7008908768F169
:103EE300BB048012E52B908768B40106F1BB240262
:103EF3008004F1BB2403FD908400EFF0A3EDF0EF09
:103F0300D3947F4006908400747FF0EDD3940740F0
:103F1300069084017407F0227872E6FE08E690D8D2
:103F23000475F00A1209FBEE75F00AA42583F583E4
:103F3300E0FCA3E0FDA3E0FEA3E0FF22E4FBFD7CA5
:103F4300607F0351FCE4FB7D017C607F0351FCE453
:103F5300FB7D027C607F0351FCE4FB7D037C607F7F
:103F63000341FC752EFF752F007530067531FF7503
:103F7300321E7533AEE4FB7D1E7F01B150752EFFFB
:103F83002212000EEF75F006A4FFC3743B9FFD756C
:103F93002EFF752F147530877531FF2290876AE0E5
:103FA300FFA3E0FEC39F222DF582E5833CF583EE5C
:103FB300F090876BE004F022E0252CFFE52D2290A2
:103FC300876CE004F0E022908767E02402F582E446
:103FD3003484F583E02290655574AAF0906AAA743C
:103FE30055F090655522E58335F0F58322852A82C5
:103FF300852983E022FD5420FCED5480FA228C6550
:104003008D66E4FEFDBF010A127CD9118E902AAAA7
:104013008022BF020A127CC9118E904AAA8015BF62
:10402300030A123FD9118E906AAA8008123AAD1181
:104033008E908AAA7455F08566828565837430F004
:10404300856682856583E0F1F7BB80047E01800588
:10405300BA20027D01EE7003EA60E5ED6401702889
:10406300AB04530380BB80027E01BF01059025553D
:104073008013BF0205904555800BBF03059065551E
:10408300800390855574F0F0AF06227480F074AA13
:10409300F0228C298D2AE4FEFDBF010A127CD9117E
:1040A3008E902AAA8022BF020A127CC9118E904ADE
:1040B300AA8015BF030A123FD9118E906AAA8008FD
:1040C300123AAD118E908AAA7455F0852A828529F9
:1040D300837430F0123FF0F1F7BB80047E0180055A
:1040E300BA20027D01EE7003EA60E9ED64017028F5
:1040F300AB04530380BB80027E01BF0105902555AD
:104103008013BF0205904555800BBF03059065558D
:10411300800390855574F0F0AF06228E278F287C9C
:10412300407D007F0211957C407D00908839317C71
:104133007C407D0190883A317CE47873F608F6AED2
:1041430027AF287C007D0A1207A8C37874E69F185E
:10415300E69E50247E40E6FA08E6FB2402FD744006
:104163003AFC74002BF58274D83AF583317C787469
:1041730006E61870010680C722E0FB7F02023AFCC4
:10418300908839E0FAA3E0FBC39433EA9403400236
:10419300412290882F123F3390D800127F2CF1BC1C
:1041A300F5831209EF908833123F3390D804127FBE
:1041B3002CF1BCF5831209EF908837E0C374809427
:1041C30080500B125F6CAF05ED24B4FF800890881C
:1041D30037125F6CAF05127F2390D80875F00A126F
:1041E30009FBECF1BCF583EFF090D809125FF1F114
:1041F300BCF583E4F090883AE004F07006908839C7
:10420300E004F0908839F119F1687531FF75321EB9
:104213007533BD7B02123F7C1248B97F0A8017F1C8
:1042230020F1687531FF75321E7533C87B02123F6A
:104233007C1248B97F187EB0124B927F407E4B7D33
:104243004C7C00024DCA7E887F231267D57A317B6E
:104253009EE4F52CFDFF127F46F1D8E493787AF6BD
:10426300F1D874019308F6E47879F67979E7C3789D
:104273007B9640026122E47878F67878E6FFC3788B
:104283007A964002611DE52C701DE5282FFFE4336B
:10429300FE18E6FD2529F19DF1EEC083C082F140B1
:1042A300E493FFEC4F8032E52C64017014127DFF20
:1042B300F19DF1EEC083C082F140E493FFEC5F8097
:1042C30018E52C64027019127DFFF19DF1EEC08395
:1042D300C082F140E493FFEC6FD082D083F080354D
:1042E300787AE6FF18E6F98FF0A4F1D8A3A3258224
:1042F300F582123FE918E6FFF15EE493FEEFFDE578
:10430300282DFDE433FCE52929F19D2DF582E58374
:104313003CF583EEF0787806417D787906416EE5C9
:1043230028787A26FFE5290826FD023EFA3008029E
:10433300815F90875DE004F0E0D394034002E4F0F2
:10434300124F3B7A347BCF752C037D047F05515983
:104353007871766E7871E6FFD3947850157B017D82
:104363000391757871E6FF7B3F7D07917578710640
:1043730080E2787176037871E6FDD3940650157B5D
:10438300FF7F6E91757871E6FD7BFF7F789175787D
:10439300710680E290875DE07027752EFF752F16FA
:1043A3007530A0F1C3916D7D037F28916B7D047FF0
:1043B30041916B7D057F32916B7D067F4DB11D4031
:1043C300E490875DE064017029752EFF752F1675E3
:1043D30030A7F1C391607D037F48916B7D047F37E4
:1043E300916B7D057F30916B7D067F3F5159B129DC
:1043F30040E290875DE064027027752EFF752F16EB
:104403007530AEF1C3916D7D037F37916B7D047F72
:104413004C916B7D057F41916B7D067F52B11D40B1
:10442300E490875DE064037033752EFF752F167576
:1044330030B5F1C391607D037F2D916B7D047F4A7D
:10444300916B7D057F43916B7D067F365159787162
:10445300E6FF7BFF7D049175B11F40D8227A347B40
:10446300BD752C037D027F5051597A347BBD752C69
:10447300032275F080EDF1A02FF160E04BF02212E2
:104483004F3B787376037873E6FFC3947D50127BBA
:10449300017D01F13AFF7BE07D069175787306801B
:1044A300E5787376027873E6FDC3940650207BFFAC
:1044B300E4FFF13AFD7BFF7F7FF13AFD7BFF7F7ED7
:1044C300F13AFD7BFF7F7D917578730680D77BFF83
:1044D3007D01E4FF91757B3F7D06E4FFF1E77F01FA
:1044E30091757B607D067F01F1E77F0291757BE02B
:1044F3007D067F0291757BFC7D017F7FF16F7F7F5E
:1045030091757BFE7D017F7EF16F7F7E91757BFFD1
:104513007D017F7DF16F7F7D817551597871E6FF54
:104523007BFF7D0591757871E6FF7BFF7D069175B5
:10453300787106E6D39478227A2F7B10752C03E4E6
:10454300FD7F6251599087E8E0F47002C159E0FFA2
:10455300740BD39F501BE0C3942150157A307B34E6
:10456300D15A7002C159752EFF752F1675304AC185
:104573004C127F0F5022E0C39438501C7A2F7BAC2F
:10458300752C037D017F6BD1617002C159752EFFBC
:10459300752F16753050C14C127F05501BE0C39424
:1045A3004E50157A307B12D15A7002C159752EFFC5
:1045B300752F16753056C14C127EFB501DE0C39407
:1045C3006550177A2F7BCEF1DFD1617002C1597527
:1045D3002EFF752F1675305C806F127EF15019E037
:1045E300C3947B50137A307B78D15A6069752EFF60
:1045F300752F167530638051127EE75019E0C3940E
:104603009250137A2F7BF0D15A604B752EFF752F82
:10461300167530698033127EDD501BE0C394A850B9
:10462300157A307B56F1DFD161602B752EFF752F24
:104633001675306F80137A2F7B8AF1DFD161601694
:10464300752EFF752F167530759087E8127E727D73
:1046530061E4FF123D5022752C037D017F6951599E
:1046630090880BE0640222127F23D39400EC940021
:104673005002C1FA90882DE0B50608A3E0B5070300
:104683001271FAED6F7002EC6E6043EF64014E60DD
:104693003D124FF77871125F79125FE8E09E402E6A
:1046A3007C007D0A1207A874002FF974D83EFA7BA8
:1046B30001C00174F62FF974D73EA801FC7D01D027
:1046C30001126398787206E61870010680C6908816
:1046D3003AE024FFF0908839E034FFF0F119F168F3
:1046E3007531FF75321E7533CC7B02123F7C124845
:1046F300B97F0B5139801CF120F1687531FF753298
:104703001E7533D37B02123F7C1248B97F1851398F
:104713007F00227F0122E0FEA3E0FF311E91827A17
:104723002E7BEE752C037D027F0A5159908400E0A5
:104733002405FD752EFF2291757873E622E0FC08AF
:10474300E6FFED8FF0A4852B82852A83A3A3258220
:10475300F582E58335F0F5837878E62582F582E402
:104763003583F58322752F1E7530332291757BFFB8
:104773007D06222582F582E43583F583740193FE59
:10478300EFFDE52C2DFDE433FC908768E07A002DE6
:10479300FDEA3CFC90876CE0252D75F080A4240095
:1047A300F582E5F03480F583E58222E6FE08E690A3
:1047B3007FFE75F00A1209FBEE75F00AA425832229
:1047C3007531FF75321E75334DFBFD7F01123D5070
:1047D3007871766E22852B82852A8322752C037D40
:1047E300017F6A2291757B017D01222FF582E5838A
:1047F3003EF58322FCFB5420FA53038022C2AFD23E
:10480300A8C2B8C289D2885389F0438902758CAD96
:10481300E4F58AD2B9D28CD2A9F5C8D2BD75CD63DD
:1048230075CB6375CCC075CAC0D2ADD2CAC299C2AA
:104833008E43878053890F438920758DECD28E90E8
:10484300851FF0908520F0759850C299C298D2AC1C
:10485300D2BC75913075950343972075948875B1D3
:104863000875B20775B30875B40775A131D2AF43A4
:10487300A71022908812125CDF90880E12768411A2
:10488300B21276CD127DF0F075E10275EA3875EA61
:104893001875EC0C75EB2875E6BA75E6BE75EB2258
:1048A30075E9BF75EE80F5E875B70143A701227F6F
:1048B300011260738022752F1E7530367531FF75B6
:1048C300321F7533F7908839E0F534A3E0F5357B73
:1048D300057D05E4FF123D50E4FF12608DE4787519
:1048E300F67875E6FFC39408504E12609BE4787621
:1048F300F67876E6FFC394805039EFC394405009AD
:10490300C2C5D2C4EF7011800BD2C5C2C47876E69B
:10491300B44005E4FF1260ACD297C2C2D2C6787627
:10492300E6FF18E612479D2F124760E012609408D5
:104933000680BE78750680A9221270BD9087B8E004
:10494300FFA3E004F0C39F4002E4F0127140FF9024
:1049530087B9E0FE044F9000E0F0D2AFEE25E024EB
:10496300A8F582E43487F583E0FFA3E09087B6CF10
:10497300F0A3EFF0F13B126168EF4E6023D21DC24A
:104983001EC21F7E877F927C887D2F12676F718E78
:1049930012687511DB90879BE0FF12720220B7FD4E
:1049A3009087A6E07002A3E06061301D5E201E299F
:1049B3007A877B927D167F2C7E0151156014E4511A
:1049C3001E600FD21E12688390879BE0FF127257FE
:1049D3008023E4511E701E8019201F197A877B9251
:1049E300510F6009E4511E6004D21F8008E4511E78
:1049F30070031271A87A877B92127DE2E4511E60E4
:104A030004511C70031271A8126875227D5A7F0F1E
:104A13007E00711678711209E374FFFFFEFDFC78C6
:104A2300711209C6C30209861270BDF13B90882D2D
:104A3300E07002A3E0700C125DC990882DEEF0A324
:104A4300EFF022201B507A887B237D167FBC7E02E9
:104A53005115603BE4511E6036D21B123F66752F21
:104A63000075300612672A7533B8123D4A1242495F
:104A7300718E90879BE0C4540F75F00AA41272A63E
:104A830095F040067F097EB0719230B74A80FBE40F
:104A9300511E7043803E201C227A887B237D167F23
:104AA3002C7E015115600DE4511E6008D21C718EDD
:104AB300718E8023E4511E701E8019201A197A8882
:104AC3007B23510F6009E4511E6004D21A8008E46D
:104AD300511E70031271D990882DE07002A3E0601B
:104AE300167A887B23127DE2E4511E6007E47FFF80
:104AF300511F70031271D9301B18123F66752F00B6
:104B030075300612672A7533B8123D4A12424912AC
:104B13006883228E27127F46E4FFFEFDFC127E3758
:104B23001260D8127E3712648F788EA607E6FFF4E0
:104B33006053908837E0FBAD29125EE5EF604312C6
:104B43007F19F5831267A25009125F70ED24B4FB3D
:104B5300800A127F19125F6AAF05AB07788EE6FFF2
:104B6300AD29125EE5EF6017AE27AF28E4FCFD78B0
:104B73008A1267685005788A0209AA74FF8007E4DD
:104B83008004E48001E4FFFEFDFC227F1D7EB03043
:104B93000214D374189F74B09E500BEF941EEE94BE
:104BA300B050037F00227876A60608A60720B7FD3B
:104BB300D2B5C2B4C2B60000E47875F6126776EED9
:104BC30030E704D2B48002C2B4C2B5EF25E07977EE
:104BD300F7EE3319F70000D2B50000787506E6B496
:104BE30010DAC2B40000D2B630B7FD7F012290883C
:104BF3003BE0FF20E70520E602A13FF13B90883B25
:104C0300E0FDC4540F90883FF0ED30E71220E40735
:104C130020E5045430600890883F7408F0C2209067
:104C2300883BE0540F90883DF0700204F07A317BAA
:104C33009E752C03E4FD7F02124259B14075321D6B
:104C4300753394E4FB7D26123F7CB14375321D75A9
:104C5300339AE4FB7D647F01123D50300117752EBA
:104C6300FF752F1D75309D126F10E0FD126ED98EEA
:104C7300318F32800C752EFF752F1D7530A4126E87
:104C8300F3123D4A90883FE024FB7002A1131460A5
:104C93005B146030146002A13BB14075321D753363
:104CA300ABF1E3123F7EB14375321D7533B17B0423
:104CB3007D487F02123D50202006F1EAD220807207
:104CC300B14D806EB14075321D7533B5F1E3123FBE
:104CD3007E127D997D6E7F02123D5020200A7F2136
:104CE3007EB07192D2208002B14D8046B1407532C0
:104CF3001D7533C1F1E3123F7E127D99127F582057
:104D0300200A7F207EB07192D2208002B14D802292
:104D1300B14075321D7533C8F1E3123F7E127D99A0
:104D2300127F5820200A7F1F7EB07192D22080020A
:104D3300B14D11DBF121A1CAF13BC22022752EFF37
:104D4300752F1D7530917531FF227F1B7EB06192E7
:104D5300752EFF752F177530A87B017D13E4FF12A5
:104D63003F7E752F177530B17B027D117F02123F95
:104D73007E752F177530B97531FF75321F7533A8DE
:104D83007B057D1C11D6200210B14D7F0C7EB071C6
:104D9300927FC07EC67D2D80067F807E847D1E7CB3
:104DA30000B1CA90883EE0600E7F1FB1BE7F20B184
:104DB300BE7F21B1BEF1EAF168E13B7EB071927F23
:104DC300807E847D1E7C008F2B8E2A8D298C28E487
:104DD3007F207E4EFDFCAB2BAA2AA929A828C3124B
:104DE30009864024E47B207A4EF9F8AF2BAE2AAD36
:104DF30029AC281208E69088061209EF908806125B
:104E03003F33EC4D4E4F70F4221267AC9087E6E0CF
:104E1300300111FCA3E0FD126ED9127F5F126EC741
:104E2300F1F7800A127ED390880CE0127EA9127FDC
:104E33003D604C127E9E4043201846D3ED944AECCD
:104E430094015033F1D4127E7E123F7CF1D9127C4F
:104E5300E9400CF1F07530A0127D627D5C80051293
:104E63007D577D607F01123D5011DBF11BF119F17C
:104E730019B1CAD218800AC2188006C2188002C2A9
:104E8300187F01228F271267AC9087E6E030011B61
:104E9300FCA3E0FD126ED9127F5FE527C4540F7E99
:104EA30000540FFF126ECEF1F7800B127ED3E5276D
:104EB300C4540F127EA9127F3D6056127E9E404D50
:104EC300201950D3ED942CEC9401503DF1D4127E73
:104ED3007E123F7CF1D9127CE9400CF1F07530A0D1
:104EE300127D627D5C8005127D577D607F01123DDE
:104EF3005011DB7F1AF11DB1CA7F1AF11DB1CA7FB0
:104F03001AF11DB1CAD219800AC2188006C21980CB
:104F130002C2197F0122B1CA7F1B7EB071927FC08A
:104F23007EC67D2D7C0022F583E4740193FA74021E
:104F330093F9120A3D120026E47876F6E47875F6C2
:104F43007875E6FFD3947F500F08E612479D2F1222
:104F53004760E4F0180680E8787606E6B408DDE4F6
:104F6300FDFF023EFAE4F527902EA8127E667A2E04
:104F73007BA8127F35127F6F40EE11DB1237DDE421
:104F8300F527902EB5127E667A2E7BB5127F35E417
:104F93007FD07E07FDFCB1CA11DB127F6F40E37542
:104FA3002EFF752F177530C07531FF75321F75339E
:104FB300B47534FF75351F75368F7B057D1711D694
:104FC30020020B7F007EB0719230B70480FBB1C228
:104FD30022F13B752EFF752F167530407531FF2278
:104FE3007B04E4FD7F02227F227EB06192752EFF57
:104FF300752F17227871A60608A60722C0E0C0F015
:10500300C083C082C0D075D000C000C001C002C040
:1050130003C004C005C006C007C2A878AA76002052
:10502300B20878AAE6D3942340F578AAE6D394236A
:1050330050211173EF601C1173EF60171173EF6050
:10504300121173EF600D1173EF600811B690883E73
:105053007405F0D2A8D007D006D005D004D003D071
:1050630002D001D000D0D0D082D083D0F0D0E032B3
:10507300E478AAF630B20878AAE6D3942340F57808
:10508300AAE6FFC3940E4028EFD394145022E4F60B
:1050930020B20878AAE6D3942340F578AAE6FFC3A2
:1050A30094004009EFD3940650037F01227F00222E
:1050B3007F0022E4FF7E01FDE478AAF630B2127885
:1050C300AAE6FCD394235009EC942340EF7EFF809F
:1050D300EBEF25E0FF78AAE6FCC3940B400BECD37F
:1050E300941150054307018013ECC39404400BEC67
:1050F300D3940A50055307FE80027EFFE478AAF694
:1051030020B20878AAE6D3942340F578AAE6D3948C
:105113002340027EFF0DED6408709DEEF460109055
:10512300883BEFF0E0C4540F7002C2207F01227F5E
:10513300FF22C0D075D008C28C78AA06D28CD0D0FA
:1051430032C0E0C083C082C0D075D01030981EC278
:105153009890851FE02401FFE433FE908520E06FE3
:105163007001EE600890851F3179E599F0D0D0D0B9
:1051730082D083D0E032E0FF04F074212FF582E483
:105183003485F58322908520E0FF90851FE0C39F3F
:1051930070037FFF22C2AF9085203179E07872F6E9
:1051A300D2AFE6FF2231887871EFF6F4600FE6FFA5
:1051B300600B908621E0FE04F031E2EFF07871E6B7
:1051C300FFF46006EF6003B40ADB908621E0600C15
:1051D3002421F582E43486F583E0FF227FFF2274E5
:1051E300222EF582E43486F58322125FD7908765F9
:1051F30004F0908621E024FBFF908765E0FEC39FC7
:105203005015A3E0FF31E2E0FEEF6E908766F09069
:105213008765E004F080DB908766E0FF1276A59057
:105223008621E0241FF582E43486F583E0B5071C6C
:10523300908766E0FF1276B7908621E0241EF58200
:10524300E43486F583E0B507037F01227F002278EB
:105253007176FF752AFF752B00752C49752D007526
:105263002E067B017A867922121CE6EF701931ED46
:10527300EF60145194EF600B78717606201608F1F5
:10528300398004E47871F6E4908621F07871E6FFC2
:1052930022E4FFFEFDFC787212615F787612615F93
:1052A300787A1209E37E867F22127E29B106127E66
:1052B30029B1251203EA9087651209EF90876512D9
:1052C3003F339087D71209EF127E52A6079087D7F4
:1052D300123F3390875E1209EFF1E9F89087D712F6
:1052E3003F331208E6908763EFF0E070037418F021
:1052F300B1A99087D7123F331208E6F1E1AF0590C9
:105303008764EDB1A89087D7123F331208E69087E0
:1053130062EBF078A6E6FE08E6FFB18A908769B1F2
:1053230017B19F126EE5127E0EC00078721209AAA1
:10533300D000F1F078761209AAE41203AC12678662
:1053430012018812677E1202911218127BCE7A63C1
:1053530079DE7842120188127DB1120291B19F1257
:10536300018890872D1209EF127E1C12085BC0047E
:10537300C005C006C00778721209AAD003D002D0B4
:1053830001D000126F3B127E94C004C005C006C05A
:1053930007127DA8120188D003D002D001D00012D9
:1053A300009790876AB17990876EB117B19F126E9B
:1053B300E5127E0EC00078721209AAD000F1F01235
:1053C3007E1C12085BC004C005C006C007787212B9
:1053D30009AAD003D002D001D000126F3B127E94F1
:1053E300C004C005C006C007127DA8120188D003FF
:1053F300D002D001D00012009790876FB1799087C7
:1054030073B1171203EAAD07AC06E41203B17B18BC
:105413007A0979ED126EE3908774EEF0A3EFF04E04
:10542300600BE02405F0908774E03400F0127E52A4
:10543300A607B10678A6A60608A607908774E070AB
:1054430002A3E0700A9087E8E0908776F0802778DF
:10545300A4E6FE08E6FF78A7E624FFFD18E634FF7E
:10546300FCB13F1267B77C017D681207BAECC31326
:10547300ED13908776F078A6B1191203EA90877737
:105483001209EF90876EE0B4530F90876A123F338F
:1054930012039B90876A1209EF908773E0B4570F4A
:1054A30090876F123F3312039B90876F1209EFC2ED
:1054B30008908769E06441704778D77C877D017BDA
:1054C300017A877965FE7F1612072A9087DC123FDF
:1054D3003390882F1209EF9087E1123F339088337E
:1054E3001209EF9087E8E0908837F0E4A3F0D20840
:1054F3009087D71266F4F1F8123F33B1B07F0122DF
:105503007F00220FEFAC0670010E14F5828C83E04E
:10551300B42CF022F008E6FE08E6FF78A4A60608FD
:10552300A607B10678A6EEF6FC08EFF6FD78A4E62A
:10553300FE08E6FFED24FFFDEC34FFFC8E278F28E9
:105543008C298D2A787B7C877D017BFF7A367915C0
:105553007E007F0F12072AC3E52A9528FFE52995C8
:1055630027FEAA27A9287B01787B7C87127C277AD0
:1055730087797B021D491209EF78A6E6FE08E6FF4C
:1055830078A4A60608A607B10678A6A60608A60765
:1055930078A4E6FE08E6F5828E83E022E4FBFA793E
:1055A3007A784422EFF0E47B64FAF9F822126FE987
:1055B300B1A91208E6EB24D0FEEA34079087EDF098
:1055C300A3CEB1A8126A661208E6F1E19087EFED67
:1055D300F1E8F8126A661208E69087F0EFF1E8F84E
:1055E300127DB99087F2B1A7127DB9F1E19087F3EB
:1055F300EDB1A8127DB99087F4EBF0127DC5540389
:10560300701EFC7D641207BAED4C700E127DC57CD2
:10561300017D901207BAED4C70069087F6741DF069
:105623009087F2E0F9FF3395E0FEAD2FED3395E07F
:10563300FCEF2DFFEE3CFEC3EF9418EE64809480E4
:105643004029127D6CFD9087F0E004F0D39D401358
:105653009087EFE004F0A3E0FD127D6CFCED8CF08D
:10566300127F679087F2E0252F802A126540502B26
:105673009087F0E014F0940050139087EFE014F05B
:10568300A3E0FF127D6CFEEF8EF0127F679087F22E
:10569300E0252F241875F01884800AE52F2975F06A
:1056A30018849087F2E5F0F09087EDE0FAA3E0FB31
:1056B3007C017D6DFFAE021207A8AC06AD07EBAE11
:1056C300027802CEC313CE13D8F92DFBEC3E127D24
:1056D300C4F1E1C3EB9FFBEA9E127DC47C017D9084
:1056E3001207BAEF2BFFEE3ACF2494CF34FEFE7CA1
:1056F300007D071207BA9087F1EDF0787E7601906E
:1057030087EFE0FF787EE6FEC39F501674F42E12F7
:105713007D72FF9087F1E02F75F00784E5F0F006C6
:1057230080DD9087F1E014FF9087F0E02F75F0079C
:1057330084A3E5F0F022301602E1E0124F3BD216CB
:105743009087D71266F4F1F8123F33B1B090882FE7
:10575300123F3390874D1209EF908833123F3390F5
:1057630087511209EF90882F123F33908743120914
:10577300EF908833123F339087471209EF126FF28D
:105783009087D7123F339087221209EFF1E9F890FF
:1057930087D7123F331208E6908729B1A79087D79E
:1057A300123F331208E6F1E1AF0590872AEDB1A865
:1057B3009087D7123F331208E6908728EBF0908743
:1057C300F2E0908726B1A8908722123F331208E6B1
:1057D300F1E1908727EDF0126FD0124F3B227C004E
:1057E3007D640207BAF0E47B107A27F9221208E6F7
:1057F30078760209E3F52E8E2D8D2C8C2B90880361
:10580300E0F52F9087E922C0E0C0F0C083C082C0DA
:10581300D075D008C2CF908804E4F0E5C0F45403F7
:1058230025E025E0FFE590F454034FF0E0FF908876
:1058330011E0FE6F6021EF600E90880FE4F0908717
:105843002004F0A374F4F090880FE0C39496502FD3
:10585300EE602C42228028EE60259087207401F0B0
:10586300A374F4F090880FE0FFC394965002800C69
:10587300EFB4960BD214EE422290880FE004F0901E
:105883008804E0908811F0908720E07002A3E06024
:105893000E908721E024FFF0908720E034FFF09002
:1058A3008801E004F0E0C394324004E4F0D20C90A9
:1058B3008806123F33EC4D4E4F601C908806A3A31D
:1058C300A3E024FFFFEE34FFFEED34FFFDEC34FFD5
:1058D300FC9088061209EF90883EE0600214F0D035
:1058E300D0D082D083D0F0D0E0327F01123D50750A
:1058F3002A017B7FE4FDFF7874A6077874E6D39BC7
:10590300503CE52A701771B61247A02F124760E08A
:10591300440271F2124760E04440F0801CE52A64BF
:10592300017016787471B61247A02F124760E0F425
:1059330071F2124760E0647FF078740680BD223014
:105943001102414590841BE0600241459087D4F0E9
:105953001274DA75321F75330DE4FB11EDE47872BE
:10596300F651565042EF75F003A424BFF582E43498
:1059730087F583E0FD71C5E0FC514675F011A42461
:10598300F2F97415F1AD123D507872E6FF5147FEFE
:105993009087D0E0FDEEB5050971C5E0FB12739E5B
:1059A300F1C078720680BAF1BB30133B71999087CE
:1059B300D0E0D39400402CE014F0E47872F6515612
:1059C300500E514671BDB5060271A778720680EE7E
:1059D30071A0600FE47872F651565007514614F0E7
:1059E3000680F5C213803C30123971999087D0E05C
:1059F300C39402502CE004F0E47872F65156500E32
:105A0300514671BDB5060271A778720680EE71A08A
:105A1300600FE47872F651565007514604F0068041
:105A2300F5C2122010022142120026124F3B90872A
:105A3300D0E075F003A42437F582E43416124F2A1C
:105A4300214222EF75F003A424BEF582E43487F5E6
:105A530083E0227872E6FFC394032230110261804F
:105A630090841BE060026180908720E07002A3E0D5
:105A730070026180E49087D4F0123F9275321E75F4
:105A830033D8FBFD7F01123D50E47871F67871E65F
:105A9300FFD3947F500C7B407D01124475787106CF
:105AA30080EBE47871F671915037EF71E3FDEF719C
:105AB300D4FC718175F011A4248CF97415F1AD1225
:105AC3003D507871E6718271AEB50610E6FE71E362
:105AD300FFEE71D4FD752A017B7F11FA7871068080
:105AE300C51248DB30133B71999087D1E0D3940002
:105AF300402CE014F0E47871F67191500E718171CD
:105B0300AEB5060271A778710680EE71A0600FE44E
:105B13007871F671915007718114F00680F5C21304
:105B2300803C30123971999087D1E0C39405502C91
:105B3300E004F0E47871F67191500E718171AEB5A5
:105B4300060271A778710680EE71A0600FE4787188
:105B5300F671915007718104F00680F5C21220108E
:105B630002415E120026124F3B9087D1E075F0038D
:105B7300A42425F582E43416124F2A415E22EF75E0
:105B8300F003A424C7F582E43487F583E022787117
:105B9300E6FFC39403227F197EB0024B929087D411
:105BA300E06401229087D47401F022FF9087D1E052
:105BB300FEEF22E6FF75F080ED22FF9087D0E0FE36
:105BC300EF22EF75F003A424C0F582E43487F58354
:105BD3002275F003A424C9F582E43487F583E02217
:105BE30075F003A424C8F582E43487F583E022F03A
:105BF30075F080EDA42480F582E5F03480F583E52B
:105C0300822F22300813A210B014500D9087E8E0C1
:105C1300F46004719991E7C210A211B014500A12F2
:105C23000026124F3B515E800FA2137212500CC21A
:105C330012C213124F3B9141124F3B020026908434
:105C430000E0FD124FD675321E75333CE4FB11EDB7
:105C5300F1FA30100281DB90841BE0707B90872087
:105C6300E07002A3E06071301214908812E0C394D4
:105C73000A5004E00491DC124B8EC21280153013DB
:105C830012908812E0D394004004E01491DC124B8C
:105C93008EC213752EFF752F16753043908812121E
:105CA3007678123F7C752F1675304812769378718B
:105CB300F67871E6FFC3940A501990881212766D34
:105CC30050067A2E7BD880047A2E7BC2F1C7787176
:105CD3000680DE1248DB815522F0D209E09035FFC1
:105CE30093F5A222908839E07002A3E07002A19C90
:105CF300F1D7F1DF908765E0FCA3E0FDC39FEC9E45
:105D03004002A19C90D800F1F1123F2B7BEF7AA4C3
:105D1300797878BF120097B1BA74F01203304069F2
:105D2300B1A390D800123F247BEF7AA47978783F0F
:105D3300120097B1BA74F01203306002504BB1A352
:105D430090D804123F247B7C7A3B79A578BFD1DEBF
:105D5300B1BD74F01203304030B1A390D804123FA8
:105D6300247B7C7A3B79A5783FD1DEB1BD74F012F8
:105D7300033060025013908766E02401FF9087652B
:105D8300E03400FE12466A8013908766E004F070E8
:105D930006908765E004F081F5124183E4FEFF225B
:105DA300908765E0FEA3E0221209FBEE75F00AA4DA
:105DB3002583F5831209B690882FE0F8A3E0F9A3B1
:105DC300E0FAA3E0FB22908839E07002A3E07002BE
:105DD300C1D7E47875F608F67875F179F1E8E09EB5
:105DE3005002C1D790D80075F00AEF123F27F1A6F1
:105DF30078C1120097B1BA74F01203305002C1CDCA
:105E03007875F182123F24F1A67841120097B1BA56
:105E130074F012033060044002C1CD7875123F1D47
:105E23007B927AB1790978C2D1DEB1BD74F01203E5
:105E3300305002C1CD7875123F1D7B927AB179093A
:105E43007842D1DEB1BD74F01203306002507B782A
:105E530075F1821247B5AF82FE7C887D2F12648F65
:105E63007877A607E6FFF46061F18A605D7875E6EE
:105E7300FE08E6FF90D8081247B5F583E0C37480A7
:105E83009480501490D80875F00AEF1247B8F16A5D
:105E9300AF05ED24B4FB800D7875F1CF1247B5F152
:105EA3006AAF05AB077877E6FFF18F601D7875F170
:105EB300821247B5FAA9827B0178237C8812639604
:105EC300E490882CF0787602678F787606E618706F
:105ED3000106A1DB1271D9E4FEFF2212009790881C
:105EE30033228F2CAA05F195C3648094805008F166
:105EF30070ED24B4FF8006F195F170AF05788FA69D
:105F030007EA252CFFE433FEC3648094805008F134
:105F130070ED24B4FF800BE52C2AFFE433FEF1700F
:105F2300AF057890EFF618E6FEB507037F012278F8
:105F330090E6FFEED39F401B18E6D39B5006EBC3BE
:105F430094B44009E4D39B5007EB9F50037F012295
:105F53007F0022788FE6D39B500A08E6FFEB9F5021
:105F6300037F01227F0022F583E0FF7E007C007D1A
:105F7300B402080F7876E6FE08E6FFD3227872E6CD
:105F8300FE08E690D80022908837E0FB7D16D1E525
:105F9300EF22EAFFC3E52C9FFFE49400FE22F58382
:105FA3001209B67B1C7A3479CF2235F0752EFFF5B2
:105FB3002F8930AB047F0122F1FA0248DB7D057F94
:105FC30001023D50752C037D05024259E6FE08E6A9
:105FD30090D80822E4908765F0A3F022908839E0F6
:105FE300FEA3E0FF2290883AE09F9088392275F063
:105FF3000AED1209FBEC22E47874F67874E6FFD319
:10600300947F500C7B807D0712447578740680EB77
:10601300787476017874E6FDD3940750177BFFE418
:10602300FF1244757874E6FD7BFF7F7F1244757819
:10603300740680E0227873A6077873E6FFD39B503B
:106043002EE52A701175F080ED1247A02F124760DC
:10605300E04402F08014E52AB4010F7873125BB6B2
:106063001247A02F124760E0F4F078730680CA222B
:10607300D29700118400EF443E900005F000C297D0
:1060830022C2C2C2C6D2C5D2C422D2971184EF445F
:10609300C0900005F0C29722AE07D2971184EE4458
:1060A300B81194908401EEF022AE07D297C2C2C217
:1060B300C6EE44401194908400EEF022E47871F629
:1060C3007871E6FFC394FA500B74222F1251E5E462
:1060D300F00680EC22F139E4FFFEFDFC788F315F9E
:1060E3007893315F78971209E3852F82852E831287
:1060F3005DBD852D82852C83123F331200937B9ADD
:106103007A1979F778411201887893F159125DBDB4
:10611300F142123F3112009390872D125DBD12019F
:106123008878971209E378971209AA71DE12018819
:10613300C004C005C006C00778931209AA71DE1215
:106143000188D003D002D001D000120097121B4A5D
:10615300F1B7788F1209E3788F0209AA1209E3E4F1
:10616300FFFEFDFC2271AF717FE0719FE408F1AF88
:106173007186081209E371867882315F7886120985
:10618300E371E7787AEEF608EFF6D39414EE940011
:10619300500471AF8009787BE624EC7977F1317193
:1061A3007FE0FF24ECFDEE34FFFC787AE6FA08E6A4
:1061B300FBC39DEA9C40097878A60608A607800AD7
:1061C300EB24147879F6E43A18F6717FE0FF4E7009
:1061D30002617BEB4A7002617B7878EAF6FC08EB9C
:1061E300F67876A60408F64A6006E61618700116D5
:1061F300EF6B7002EE6A6008787906E618700106A4
:10620300D37877E6940118E694004024787A12470D
:10621300AE125FA178C1120097787671C11247BCA4
:1062230071B7600C400A7877E6161870011680D0B3
:106233007878125F799087B7E09F9087B6E09E40A9
:1062430021081247AE125FA1784112009778787146
:10625300C11247BC71B7500A787906E61870010677
:1062630080CEF176787AA60608A607787A125F7947
:10627300787996EE1896506A907FFE75F00AEF12C1
:1062830047B8718D7E877F9C7C887D2F11D8787E5F
:106293001209E37E877F9CF14CF4603C125F8A60B5
:1062A300379087A4F1A25009125F70ED24B4FB80EC
:1062B3000A9087A4125F6CAF05AB077875E6FF12EF
:1062C3005F8F601471A7124A24400D71A71209E36E
:1062D300787AE6FE08E6719F787B06E61870010679
:1062E3008089787DE618467002617BE47F207E0317
:1062F300FDFC7882F1684002617B787C1247AE71C5
:106303008D7A877B9C7D0F7FBC7E02124B1678862D
:106313001209E371867886124A24605CE4FFFEFD6D
:10632300FC7886124A2460509087B9E0FFE4FCFDB4
:10633300FE7BCC7A0CF9F812085BEF787D26FFEE32
:106343001836FE787AF608EFF69087A6E06E7003AB
:10635300A3E06F6023787AE6FF08E69087A6CFF084
:10636300A3EFF07A87799C7B0178927C8771969072
:1063730087A6E0FEA3E0FF22E4FEFF229087B6E0BB
:10638300FEA32274FFFFFEFDFC22FAA9827BFF78A5
:106393009C7C877D017E007F0A02072AFF08A606F0
:1063A30008A60722787E1209AA78822278767600D8
:1063B30008760122F5831209D374F0020330E6FA5A
:1063C30008E6907FFE75F00A1209FBEA22E0FF7EE1
:1063D300007C0E7D101207A8E4FCFDA804A905AA01
:1063E30006AB0722E4788AF608F6717FE0FF24FF04
:1063F300788DF6EE34FF18F6EF4E7002818B788CB1
:10640300E6FE08E6FF788AE6FC08E6FDD39FEC9EED
:106413005072ED2FFFEC3EC313FEEF13FF788EEEA9
:10642300F608EFF608A60608F66D7002EC6E6054E7
:10643300788EE6FE08E6FF788D66700318E66E60D8
:106443004390800875F00AEF125DAB74F0120330CD
:10645300500B788FE624FF798DF13180A1788EE699
:10646300FE08E690800875F00A125DAB74F0120323
:10647300306011400F788FE62401798BF718E436EA
:1064830019F781017891E18FE4FEFF22F139852F1D
:1064930082852E83125DBD8F828E83123F3312005D
:1064A30093788FF159125DBDF142123F311200937F
:1064B30078931209E378931209AAD1BA788F120953
:1064C300AA121C73F17E120188F18612029171DE09
:1064D300E4FFFE7DE17C431200931203EA7897EE1A
:1064E300F608EFF6B140500D18B157ED2468FFECF4
:1064F3003401FE800B7897B157ECC313FEED13FF05
:106503007897A60608A607E4FFFEFDFC7893B1473B
:10651300700DFFFEFDFC788FB14770037FFF22B142
:106523004FB1407D0050027D01ED6009125F70EDB7
:1065330024B4FF8007B14F125F70AF0522C3EE642E
:10654300809480221209C674F00203307897E6FE25
:1065530008E6FF22E6FE08E6FF7C017D6802080FDD
:10656300E47872F608F6301102C1A590841BE0604E
:1065730002C1A5F1CC752F147530B2F12A7533B869
:10658300E4FB7F01123D50908839E07002A3E07074
:106593001B752A017B7FFDFF1258FA123F92753259
:1065A3001F7533BD7B047D19E4FFC15D752EFF7537
:1065B3002F147530C27873E62401F53218E436F5EA
:1065C30031E4FB7D661258ED125F80123F24D1FF48
:1065D3001203ACC00471E0125F80123F24D000D1DB
:1065E300D4125F80123F24D1CA7F53600250027FCE
:1065F3004E8F31752EFF752F147530C8D1E7F537DF
:10660300D1BC7B02D1C3123F1BD1FF1203ACC00428
:1066130071E0123F1BD000D1D4123F1BD1CA7F5768
:10662300600250027F458F31752EFF752F14753030
:10663300E1D1E7F537D1BC7B04D1C37872125FCFC8
:106643001247B5F583E075F002F19B752EFF752FA8
:10665300147530FA7B067D077F01123D50125FBB34
:10666300301317D37873E6940018E69400400708B4
:10667300E61618700116C213A169201202A16990CF
:10668300883AE024FFFF908839E034FFFEC3787333
:10669300E69F18E69E50070806E618700106C21228
:1066A300A16922908802E0FCE41203B67B857AEBB1
:1066B30079C7783D1201888F378E368D358C342219
:1066C3007D077F01023D50E4FBFAF9F874F0020301
:1066D30030120093E4FBFA797078421202919087AA
:1066E300BA0209EF9087D5E0F532A3E0F53390873E
:1066F300BAE0FCA3E0FDA3E0FEA3E022E4FBFA7909
:106703006178451202911203EA9087D5EEF0A3EF68
:10671300F09087D5E0FEA3E0FFE4FCFD7B107A0E4A
:10672300F9F812085BE4227531FF75321E22F7185F
:10673300E634FF19F7228E2C8F2D8C2E8D2F22E518
:106743002D2404F582E4352C227C887D2F918F78CB
:1067530075A607E6FF221209E3E52F2404F582E478
:10676300352EF583221209C6D302098611D8787112
:106773000209E37876E6FE08E6FF22E4FBFA7934C1
:106783007843227BDC7A0F7949784022E62401FFA3
:1067930018E436FE2275F00AA485F031F53222E0C2
:1067A300FF7E00C37480948022E47871F608F608B3
:1067B300F608F622E4FBFAF9783F1200970203EA9F
:1067C3007B017D0A7F02123D50908400E0FD752E0F
:1067D300FF22F14C908837E0D39F4012EF24B4FF9F
:1067E300E433FEE0FDC3EF9D7877F6EE800E9088EC
:1067F30037E0FF7875E6C39F7877F6E4940018F6E0
:10680300125F77740B9FE49E500FC3EF9421EE94B5
:106813000050067A337B48804F125F7774219FE4E0
:106823009E500FC3EF9438EE940050067A327BFEED
:106833008036125F77747B9FE49E500FC3EF949270
:10684300EE940050067A327BB4801D125F77749207
:106853009FE49E500FC3EF94A8EE940050067A3243
:106863007B6A80047A327B20752C03E4FD7F670208
:10687300425990879BE0FF314E7E877F921267D506
:1068830078711209AAF1E9752EFF752F1675307B01
:10689300516F7B057D4B7F02123F7E752F1675303E
:1068A30080852A348529338528328527317B067DE7
:1068B300767F01123D50E47F64313F500B752EFF0C
:1068C300752F16753082806B51661255A9D3120944
:1068D300865012E47FC8313F500B752EFF752F167B
:1068E300753088804E5166E47BC8FAF9F8D31209F3
:1068F300865014E47F2C7E013140500B752EFF75BA
:106903002F1675308E802C5166E47B2C7A01F9F8B2
:10691300D31209865014E47F907E013140500B75E9
:106923002EFF752F167530948009752EFF752F165F
:1069330075309A7B05E4FD7F02023D50FEFDFCAB02
:106943002AAA29A928A827C30209868F277A337B75
:1069530092752C037D037F67124259E527C4540FB8
:1069630030010D7E00540FFFD1CE8E318F32800364
:10697300126798752EFF752F1E7530247B037D6F6C
:10698300E4FF123D50E527540F14B40700400241C1
:106993005B90699B12724C730269B00269C602690B
:1069A300E80269FF026A16026A38026A49515C7595
:1069B30031FF75321E753370E4FB123D4C7A307B28
:1069C3009A4158515C7531FF75321E753377123F0A
:1069D30078515F7531FF75321E753370123D4A7AF7
:1069E300317B1C8070515C7531FF75321E753381AC
:1069F300123F78123D3B7A317B9E8059515C753151
:106A0300FF75321E75338E123F78123D3B7A317B10
:106A13009E8042515C7531FF75321E753394123F6F
:106A230078515F7531FF75321E75339D123D4A7A79
:106A3300317B9E8020752EFF752F1E75302BF1291B
:106A43007A317B9E800F752EFF752F1E75302FF1C7
:106A5300297A317B9E12425422752EFF752F1E75A3
:106A6300302822AF2AAE29AD28AC27228F348E33AB
:106A73008D328C31228F2712453BC39087E7E094F8
:106A83004A9087E6E09401400F90872BE0FFA3E054
:106A93009087E6CFF0A3EFF0E5276402600261AFD1
:106AA300124FD675321E75335BFBFDFF123D50301E
:106AB3000117F19FF110E0FDD1D98E318F321267AA
:106AC300C3752F167530C0800DF19FD1F31267C3C4
:106AD300752F167530C4F1C9124FD675321F753331
:106AE30097D1BF9087E8E0F47002619AE0FF740BDE
:106AF300D39F5011E0C39421500B752EFF752F16B1
:106B03007530C861A6127F0F5011E0C39438500B43
:106B1300752EFF752F167530CF61A6127F055011A4
:106B2300E0C3944E500B752EFF752F167530D6802B
:106B330072127EFB5011E0C39465500B752EFF75E6
:106B43002F167530DD805C127EF15011E0C3947B0B
:106B5300500B752EFF752F167530E48046127EE7B5
:106B63005011E0C39492500B752EFF752F1675309C
:106B7300EB8030127EDD5011E0C394A8500B752ECC
:106B8300FF752F167530F2801A752EFF752F167547
:106B930030F99087E8800C752EFF752F177530003C
:106BA3009087E8127E727D0A7F02C196E527640111
:106BB3006002A1C1124FD675321F7533717B01FD7F
:106BC300FF123D50300115752EFF752F17753007D5
:106BD300D1EB908737123F33D1FE8011752EFF75AD
:106BE3002F17753010908737123F33F152516FF1E1
:106BF3006E124FD67532207533127B02E4FDFF12FD
:106C03003F7E752F17753019908726D1F67B027D4D
:106C13001CE4FF123F7E752F177530247531FF7505
:106C230032177533319087F2E0F534A3E0F5357B05
:106C3300027D3AE4FF123F7E124FD975321F75333E
:106C43009E7B03D1C1300115752EFF752F1775304B
:106C530033D1EB90873B123F33D1FE8011752EFF6A
:106C6300752F1775303C90873B123F33F152516FAC
:106C73007B037D26E4FF123D50124FD6D1B930017C
:106C83000EF181F110E0FDD1D98E318F328004F104
:106C930077D1F37B04F1679087291263D0F1B49025
:106CA3008728E0FFE4FEEB2FF11E90873F1209EFE8
:106CB3009087631263D0F1B4908762E0FFE4FEEB48
:106CC3002FF11E90871C1209EF90873F125DBD9034
:106CD300871C1266F4C39BFFEE9AFEED99FDEC98B8
:106CE300FC9087571209EF124FD675322075330E79
:106CF3007B05D1C1908737123F33EC4D4E4F604136
:106D0300300119F195F1A9125DBD12085B90875707
:106D1300125DBD1208E6D1EBD1FE801CF18BF1A907
:106D2300125DBD12085B908757125DBD1208E6D154
:106D3300EB1208E6E41203AC516F7B057D2CE48073
:106D430010300104F1958002F18BE4F5317B057D70
:106D53002CFF123D50124FD6F1607B06D1C1127445
:106D6300CE30010AD1D28E318F32F18180091207E0
:106D7300A88E318F32F1777B06F167124FD67532C9
:106D83001F7533A27B07D1C112472F752F1775309B
:106D9300699087F0E0F5319087EFE0F5327B07E407
:106DA300FF123F7E752F177530737531FF753217DC
:106DB30075337E1266A67B077D4BE4FFC196124FA7
:106DC300D675321F753371E4FBFDFF123D50300160
:106DD30015752EFF752F17753082D1EB90873712FB
:106DE3003F33D1FE8011752EFF752F1775308A90B2
:106DF3008737123F33F152516FF16E124FD6F16064
:106E03007B02D1C190880CE0FF602A300111D1CC04
:106E13008E318F32752EFF752F177530928010903B
:106E2300880CE0126798752EFF752F177530997BC4
:106E3300037D3280137BFF7A1E796CF1D7FFC37415
:106E43005A9FFD124FD6F1E0E4FF123D50124FD688
:106E5300D1B9300121124FF07530A0F110E0FDD10E
:106E6300D98E318F327B057D2D7F02123F7E752FA8
:106E7300167530C08017124FF07530A0D1F37B0523
:106E83007D2D7F02123F7E752F167530C47B067DE4
:106E93005E7F01123D509087F2E0FF908732E06FF2
:106EA3006002F1D0F1F29087E6E0FFA3E090872B38
:106EB300CFF0A3EFF02275321E75335B7B04E4FD44
:106EC300FF023D5090880CE0FF7E007C007D0A129B
:106ED30007A8AC06AD07E41203B17BDB7AF9791E90
:106EE300783F1201880203EAE47BE87A03F9F82287
:106EF3009087E6E0F531A3E0F532221208E6E412CA
:106F030003AC7BDB7AF9791E783F0201889087E630
:106F1300E0FCA32278711209C6EF2BFFEE3AFEEDD7
:106F230039FDEC38FC227531FF75321E7533A5E44B
:106F3300FB7D197F01023D50C3EF9BFFEE9AFEEDEF
:106F430099FDEC98FC787A1209E3787A1209AAE49D
:106F53001203ACE4FBFA797A784402029175321E8B
:106F63007533F4227D32E4FF023D507B017D2CE436
:106F7300FF023D50752EFF752F1775304D22752E6C
:106F8300FF752F1775304522752EFF752F17753036
:106F93005F22752EFF752F1775305522752EFF75DD
:106FA3002F167530BC22E47F107E0EFDFC908737D0
:106FB30022A3E075F03CA4FFEB2FFBEA35F0FAEDDA
:106FC30039F9EC38F8227B027F01023D507F1E7EA7
:106FD300B0024B9212000EEF75F006A42275321E1A
:106FE30075336C7B03228F2A8E298D288C27229060
:106FF30087F2E0908732F0221270BD20080201BCB4
:1070030090882F123F3390874D1209EF90883312E7
:107013003F339087511209EF9087E6E07002A3E0B7
:10702300603F7E877F4D7C877D4312676FE47FE8F7
:107033007E03FDFC78711267685002800211BD90D7
:10704300873B123F33126F1790873B1209EF9087EC
:1070530037123F33126F179087371209EFD20F8021
:1070630038C20FA20F300E01B3502E7D007C607F1B
:107073000312409590873BE0FB7D00123F609087B1
:107083003CE0FB7D01123F6090873DE0FB7D0212F7
:107093003F6090873EE0123F5D90882F123F339010
:1070A30087431209EF908833123F339087471209C1
:1070B300EF300F03D20E22C20E22E4FFFEFDFC7856
:1070C300710209E38F27E47872F631404527F0D245
:1070D300AF7A8079067BFFC001E52775F002A4240F
:1070E300A6F9748735F0A801FC7D01D0013139314F
:1070F3002BE0FEA3E0FFF47002EEF46004EF4E70A9
:107103000B312BE4F0A3F07872F6800478727601E9
:10711300312BE0FEA3E0FF9087B7E02FF09087B616
:10712300E03EF07872E6FF22E52725E024A6F5820B
:10713300E43487F583227E007F0202072AC2AF90E0
:1071430000E0E054F822787176017871E6FFD39479
:1071530007501111C7EF60077871E69087B8F07890
:10716300710680E62278397C887D017B017A40793B
:10717300003139125FDF4E602BC3EF9433EE94037B
:1071830050167C007D0A1207A878007CD87D017B0D
:10719300017A40790202072AE4908839F0A3F0FFCC
:1071A300FE12411E22E49087A6F0A3F0C21DC21E68
:1071B300C21FC219FFFEFDFC90879231D0908796C3
:1071C3001209EF90879A74FFF0E4A3F0221209EFFB
:1071D300E4FFFEFDFC2231FAC21BC21CC21AFFFEF1
:1071E300FDFC90882331D09088271209EF90882BDB
:1071F30074FFF0E4A3F022E490882DF0A3F0225171
:107203009994004043ED604014B40700503A9072E3
:1072130017514C7302722C027230027234027244A0
:1072230002723802723C0272407F0180167F028034
:10723300127F04800E7F03800A7F0680067F07800B
:10724300027F057EB0124B922275F003A4C58325FD
:10725300F0C5832251999400403BED14B4070050CC
:107263003490726A514C7302727F0272810272858A
:1072730002729102728902728D02728D80007F0FF9
:10728300800E7F10800A7F1080067F0D80027F10A2
:107293007EB0124B9222EF540FFDEFC4540F75F0E2
:1072A3000AA4FEFFC39087E7E09F9087E6E022E40D
:1072B3007872F690880BE0F6301102618F90841B90
:1072C300E06002618F908400E0123F9175321E7579
:1072D30033E2E4FB1258ED30131290880BE0D394A1
:1072E300004005E014F0D209C2138013301210904D
:1072F300880BE0C394025005E004F0D209C2127572
:107303002EFF71977531FF75321F7533757B027DC3
:1073130005123F7C71977531FF75321F75337F7B83
:10732300047D05123F7C71977531FF75321F7533EC
:10733300877B06125FC090880BE07006719E7B020C
:10734300801890880BE0B40106719E7B04800B903B
:10735300880BE0B40207719E7B06125FC0301027D2
:10736300C21090880BE07872F6124F3B124720123E
:107373003F9575321F7533EC126FC91248DB124FFC
:1073830021124DCA124F3B125FBB41BB7872E6908C
:10739300880BF022752F1475308A22752EFF752FF6
:1073A3001475308E22908400E0123F9175321F7560
:1073B300332FE4FB1258ED125FFA20114690841B21
:1073C300E070403012069107C21280073013049117
:1073D30007C213752EFF752F157530527B037D057C
:1073E300123F7C752F157530607B05125FC020013D
:1073F30006719E7B038004719E7B05125FC0124859
:10740300DB80B722A201B39201D2092291DA126F73
:1074130060E4FB1258ED125FFA30110281C49084CC
:107423001BE0600281C430121290880CE0C39421E7
:107433005005E004F0D209C2128013301310908873
:107443000CE0D394004005E014F0D209C213752E6A
:10745300FF752F147530947B03125FC090880CE086
:10746300604D200112752EFF752F147530A491C540
:1074730091CE1207A8800E752EFF752F147530ACB0
:1074830091C5126EC78E318F32752EFF752F14750D
:1074930030A87B03123D4C752EFF752F147530B049
:1074A3007B037D0A123F7C71A17B037D6E800812F2
:1074B3003F92126FE07D087F01123D501248DB813D
:1074C3001C227B037D467F01023D5090880CE0FF28
:1074D3007E007C007D0A22908400E0FD752EFF75FE
:1074E3002F147530907531FF2291DA75321F753381
:1074F30052E4FB1258ED125FFA20114B90841BE00B
:107503007045301206B14BC2128007301304B14BE1
:10751300C213300213B15375321F75334A7534FFEA
:1075230075351E75366C8011B15375321F75334A2C
:107533007534FF75351E7536687B037D0A7F01122E
:107543003D501248DB80B222A202B39202D209223A
:10755300752EFF752F157530867531FF2291DA75FB
:10756300321F753341E4FB1258ED125FFA201164A8
:1075730090841BE0705E301214908803E0C3648033
:10758300948C5005E004F0D209C212801530131216
:10759300908803E0D3648094744005E014F0D2092A
:1075A300C213908803E0FFC364809480400D752E5E
:1075B300FF752F157530708F31800F752EFF752F66
:1075C3001575307B908803E0F5317B03126F34121D
:1075D30048DB809922301102C16C90841BE0600269
:1075E300C16C91DA75321E7533FBE4FB1258ED3032
:1075F300121490880EE0C3940A5007E004F0D209F5
:10760300D184C212802030131D90880EE0D39400E1
:107613004012E014F0D209E090360A93FFF5AA7401
:10762300FF9FF5ABC213752EFF752F1575300690AE
:10763300880ED178123F7C752F1575300BD1937856
:1076430072F67872E6FFC3940A501990880ED16DD2
:1076530050067A2E7BD880047A2E7BC2125FC778BD
:10766300720680DE1248DBA1D822E0FEEFC39E90B3
:107673008400E0FF22E075F00AA4F5317B037D4B23
:1076830022E090360A93FFF5AAC374FF9FF5AB225D
:107693007B037D647F01123D507D057F0A123EFA14
:1076A300E42253070FEFD39409EF50042430FF2251
:1076B3002437FF225307F0EFC4540FFFD39409EF8D
:1076C30050042430FF222437FF22D2B5D2B6C2B4ED
:1076D300D2C32275EAB022127DF0F0A3E0546070A9
:1076E3001BA3E024FB600E14600D24FD600B240833
:1076F300700A02002E80DC8007027C4C43EA4022A1
:10770300908819E024FE602614603324E2605C1440
:10771300606B24216002E19B127E5FA37435F0A3AA
:107723007451F0908814E4F0A37412F0806E127E0A
:107733005FA37435F0A3746DF090356F803B908830
:1077430018E075F003A424F6F582E5F03435F583EB
:10775300E493FB740193FA740293F9908820EBF09D
:10776300A3EAF0A3E9F01207508022127E5FA3740C
:1077730035F0A37464F0903563E4938010127E5F58
:10778300A37435F0A37492F0903591E493FF90883D
:1077930014E4F0A3EFF0800443EA402290881DE054
:1077A300FE90881CE0FDEDFF789EEEF6FE08EFF6F6
:1077B300908814E0FCA3E0FDC3127EBF7F0050025B
:1077C3007F01908813EFF0789E125F79ED127EBFF0
:1077D3004006A3EEF0A3EFF053EA7F908820A3E0E6
:1077E300FAA3E0F9EA497003027886908814E0FE70
:1077F300A3E0FF4E7007127894F5EA807A78A2EE40
:10780300F608EFF6D3118C400618760008760811B7
:1078130094FF78A3E64FF5EAE478A0F608F6C37977
:10782300A1E778A39618E66480F819E76480985076
:107833001F908820E0FBA3E475F001120845A9F02E
:10784300FA120750F5E778A106E61870010680CE14
:1078530078A2E6FE08E6FFC3908815E09FFD9088B6
:1078630014E09EFCF0A3EDF04C7015908813E060DB
:1078730006C3EF118C5009908820E4F0A3F0A3F025
:107883007F012275EA907F00229408EE6480948041
:1078930022E5EA648054804430228B658A668967D6
:1078A300D3ED9408EC6480948040047C007D08113F
:1078B300944DF5EAED1DAE0470011C4E600F11D11D
:1078C3007002056614F9120750F5E780E722AB65ED
:1078D3000567E567AA6622908816E0FEB4210DA32A
:1078E300E0B40908E490849DF07F0122EE64A17066
:1078F30023908817E0B4011C53EA7F7B017A8479D3
:10790300DF7D087C00119D9084DE7408F0FF12393E
:10791300CC7F01227F0022C0E0C0F0C083C082C0C0
:10792300D075D018E5E830E111E5EA30E609E5ED78
:107933005430600353EABF53E8FDE5E830E45543B0
:10794300EA3853EADF9084DEE0FFC394405040C33B
:1079530074409FFFC39408500280027F08789BEF16
:10796300F69084DEE024DF911FEFFD7C00119D5330
:10797300E8EF789BE6FF9084DEE02FF0C39440406D
:10798300049138800F9084DEE0FF1239CC8005919A
:107993006653E8EFE5E830E37BE5ED30E616514763
:1079A300789DEFF653E8F7E6606A11DAEF70651237
:1079B30076DA8060E5ED540F605490849DE0C394C3
:1079C30040504BE5ED540F789BF6087600789BE624
:1079D300FF08E6FEC39F501490849DE02E249EF57D
:1079E30082E43484F583E5EFF00680E163ED8053B0
:1079F300E8F7123933789BE6FF90849DE02FF0C3BC
:107A030094404010718B53EA9043EA20800663ED63
:107A13008053E8F7E5E830E205518853E8FBE5E8F1
:107A230030E00353E8FEE5E830E70353E87FE5E899
:107A330030E50653E8DF124887D0D0D082D083D018
:107A4300F0D0E032756501756688756716E5ED540B
:107A53000F6408600643EA407F0022E4789EF6083C
:107A6300F611D17002056614F9E5EF120796789FB7
:107A730006E618700106789FE66408184670E2432C
:107A8300ED807F0122789E760008760778A9E6903C
:107A9300878AF0C3742496FFE41896FED374079F75
:107AA300EE6480F87480984007789EEEF608EFF64F
:107AB300789EE6FE08E6FF78A8E6FC08E62422F9AD
:107AC30074863CFA7B01788B7C8791277A87798A45
:107AD300756A00756B087F017E007100789EE6FE73
:107AE30008E678A80826FFF618EE36FEF6C3EF94EC
:107AF30024EE648094804004E4F608F6228E658FB9
:107B0300668B678A68896943EB28E5666401456586
:107B13007006717F4002800CE56664024565700A59
:107B2300717F4006756A00756B08E478A0F608F665
:107B3300C378A1E6956BE56A6480F5F018E6648086
:107B430095F0501CAB670569E569AA687002056882
:107B530014F9120750F5E60806E61870010680D0FE
:107B6300E5EB648054804420FFE566640245657E4E
:107B73000070027E40EF4E456BF5EB22D3E56B942C
:107B830008E56A648094802290849EE06074B40562
:107B93000890849C7401F08022781C7C847D017B96
:107BA300017A84799E7E007F4012072A7E007F40FF
:107BB3007D007B017A84795C120A4390849EE024E1
:107BC300FD603224FD602514601914601B146009E4
:107BD30024087029E4F5AE801790841B7401F0E447
:107BE300A3F0229106E48008910F80049106910F7F
:107BF30090841CF02290849F912F124001E4FF1285
:107C030039CC2290849FE09000E0F0229084A0E0A1
:107C13009000E2F0E422518853EADF22F9E434844D
:107C2300FA7B01227D0112072A7B0122E0FFA3E0F8
:107C3300FCA3E0FD2290849CE06002E4F090841CAD
:107C4300E06005E4FF1239CC22908818E0D3940059
:107C530090881F40077404F0911980037403F07532
:107C6300EAB0221277DEEF7022908817E0B4051590
:107C7300A3E0FF4480F5EEEF90881F60057403F0E6
:107C830080037402F090881774FFF0228B688A696E
:107C9300896AE56C156CAC6B7002156B4C601D0F3B
:107CA300EFCCEECC70010E14F5828C83E0FD91C015
:107CB3007002056914F9ED12079680D622AB6805A8
:107CC3006AE56AAA692290455574AAF0904AAA7493
:107CD30055F09045552290255574AAF0902AAA7420
:107CE30055F09025552275321E75335B7B047D0359
:107CF3007F01123D507A337B9B752C037D017F50AE
:107D0300124259C37872E6946418E6940022F5830C
:107D1300740193FA740293AE02FF7875EEF608EFDE
:107D2300F6F5828E83E49390876AF0E490876CF093
:107D330022E6FF7E0090841FE02FF090841EE03E39
:107D4300F0C3908421E09FFF908420E09EFEF0A387
:107D5300EFF04E22752EFF752F177530A47871E65C
:107D6300F53108E6F5327B03229087EFE024F4F542
:107D730082E43487F583E022EEFDE52C2DFDE43328
:107D8300FC908768E07A002DFDEA3CFCD3ED947FFC
:107D9300EC6480948022752F1D7530BD90883DE082
:107DA300F5317B042278761209AAE41203ACE4FBD2
:107DB300FA7961784522AF2EAE2DAD2CAC2B02089B
:107DC300E6FA9087EDE0FEA3E0FF2290876CE08F58
:107DD300F0A4FF7875E6FC08E68C832FF582227DFC
:107DE300167F207E03124B1678710209E3908820D8
:107DF300E4F0A3F0A3F0908814F0A3227878E625AA
:107E030028FFE433FE08E6FD25292278721209E3F0
:107E13007BA07A8679017800227FA07E867D017C13
:107E23000078760209C678A6EEF608EFF678A4A6DF
:107E33000608F622788A1209E37C887D2FAF2BAEE1
:107E43002A2275321F7533937B037D44E4FF227826
:107E5300A6E6FE08E6FF78A4A6060822908820740A
:107E6300FFF022E493FFE5278FF0A4240FFF22E025
:107E730025E0F532E433F5317B052275321E753387
:107E8300627B027D032275321F75338F7B03E4FF10
:107E930022E4FBFA7970784202018808E6FC08E6DE
:107EA300FDC39FEC9E2275F00AA47871A6F008F634
:107EB30022FED3EF947FEE64809480229FEE648051
:107EC300F8EC648098227531FF75322075330822EF
:107ED300FEA3E07873A60608F6229087E8E0FF7415
:107EE30092D39F229087E8E0FF747BD39F229087F1
:107EF300E8E0FF7465D39F229087E8E0FF744ED3D8
:107F03009F229087E8E0FF7438D39F229087E8E0B0
:107F1300FF7421D39F22E52B2408F582E4352A221E
:107F2300908839E0FCA3E0FD2275F00AEB1209FB0F
:107F3300EA22752C037D060242597871E6FE08E6B3
:107F4300FF4E228F288D298A2A8B2B22908769F056
:107F530075F003A4227D647F02023D507873A60668
:107F630008A60722849087F0E5F0F0220527E5278D
:047F7300C394092288
:027FFE00111759
:00000001FF
